:020000040000FA
:100000000004040000000000041A0000081A0000A8
:100010000C1A0000101A0000141A00000C1B00003B
:100020000C1B00000C1B0000181A00001C1A00001A
:10003000201A0000241A00000C1B0000281A0000DF
:100040002C1A0000301A0000341A0000381A000080
:100050003C1A0000401A0000441A0000481A000030
:100060000C1B00000C1B00004C1A0000501A000072
:10007000541A0000581A00005C1A00000C1B000003
:10008000601A0000641A00000C1B0000681A0000CF
:100090006C1A0000701A0000741A0000781A000030
:1000A0007C1A0000801A0000841A0000881A0000E0
:1000B0000C1B00000C1B00000C1B00008C1A000025
:1000C000901A0000941A0000981A00009C1A000070
:1000D000A01A0000A41A0000A81A0000AC1A000020
:1000E0000C1B00000C1B00000C1B0000B01A0000D1
:1000F000B41A00000C1B00000C1B0000B81A000012
:10010000BC1A00000C1B00000C1B00000C1B0000A4
:100110000C1B00000C1B00000C1B00000C1B000043
:10012000C01A00000C1B00000C1B0000C41A0000C9
:10013000C81A0000CC1A00000C1B00000C1B0000A9
:100140000C1B00000C1B0000D01A00000C1B000050
:100150000C1B00000C1B00000C1B0000D41A00003C
:100160000C1B00000C1B00000C1B0000D81A000028
:10017000DC1A0000E01A0000E41A0000E81A00008F
:10018000EC1A0000F01A0000F41A0000F81A00003F
:10019000FC1A0000001B0000041B0000081B0000EC
:1001A0000C1B00000C1B00000C1B00000C1B0000B3
:1001B0000C1B00000C1B00000C1B00000C1B0000A3
:1001C0000C1B00000C1B00000C1B00000C1B000093
:1001D0000C1B00000C1B00000C1B00000C1B000083
:1001E0000C1B00000C1B00000C1B00000C1B000073
:1001F0000C1B00000C1B00000C1B00000C1B000063
:10020000FFFFFF00FFFFFF00C8040000C80400005C
:10021000C8040000C8040000C8040000C8040000AE
:10022000C8040000C8040000C8040000C80400009E
:10023000C8040000C8040000C8040000C80400008E
:10024000C8040000C8040000C8040000C80400007E
:10025000C8040000C8040000C8040000C80400006E
:10026000C8040000C8040000C8040000C80400005E
:10027000C8040000C8040000C8040000C80400004E
:10028000C8040000C8040000C8040000C80400003E
:10029000C8040000C8040000C8040000C80400002E
:1002A000C8040000C8040000C8040000C80400001E
:1002B000C8040000C8040000C8040000C80400000E
:1002C000C8040000C8040000C8040000C8040000FE
:1002D000C8040000C8040000C8040000C8040000EE
:1002E000C8040000C8040000C8040000C8040000DE
:1002F000C8040000C8040000C8040000C8040000CE
:10030000C8040000C8040000C8040000C8040000BD
:10031000C8040000C8040000C8040000C8040000AD
:10032000C8040000C8040000C8040000C80400009D
:10033000C8040000C8040000C8040000C80400008D
:10034000C8040000C8040000C8040000C80400007D
:10035000C8040000C8040000C8040000C80400006D
:10036000C8040000C8040000C8040000C80400005D
:10037000C8040000C8040000C8040000C80400004D
:10038000C8040000C8040000C8040000C80400003D
:10039000C8040000C8040000C8040000C80400002D
:1003A000C8040000C8040000C8040000C80400001D
:1003B000C8040000C8040000C8040000C80400000D
:1003C000C8040000C8040000C8040000C8040000FD
:1003D000C8040000C8040000C8040000C8040000ED
:1003E000C8040000C8040000C8040000C8040000DD
:1003F000C8040000C8040000C8040000C8040000CD
:100800000FA220000E7F24000E01880000000000CF
:10081000000020000000E000020032000001200083
:1008200020028800140007005B0007000000E000C1
:1008300003003A0080682100010020000200370018
:100840000000200001002000810F70000100320034
:1008500014000700000020000000E0000200320049
:100860000000020000000000DC1402000000000094
:100870000040DA000000FE004440A90040112000C2
:100880000000E0000300320000002000A00188000A
:100890004440A800000006008A1F78008B1F7800E3
:1008A0000000060091018800800478000000EB0041
:1008B0001A003700E284440032A0B4009905BA005F
:1008C000E284440032A0B4009906BA00E2844400F5
:1008D00032A0B4000006EB00476FDE00FD07B20057
:1008E000636CE10003003A00EBFF07000000EB003F
:1008F0000A003700606CE10004003A00005DEB0084
:100900008B05E900FDFF3E00040037006168E1004F
:10091000010032000086EB000B00070019C7BA0087
:100920001905BA000E04E00003003A000A00E000D6
:10093000E0FF3A0000000600FE07B2009E018800BA
:100940008A047800F5FF3700395DBA008B05E900AD
:100950000C003200295DBA008B05E9000800320066
:100960000C00E00003003A00E284440032A0B4002E
:10097000F5FF370019DDBA008B05E900FAFF3A00F0
:100980008904E800E184440032A0B40000000600BD
:100990000040DA000000FE00000005008001780041
:1009A00002003700815978000201E9000200E000EE
:1009B000FCFF3A00000006001201000000020000E7
:1009C0000000000000080000D80400003C00000007
:1009D0000001000001020000000100000902000007
:1009E000290000000101000000C0000032090000E1
:1009F00004000000000200000300000000000000EE
:100A0000092100001101000000010000221D00006A
:100A10000007000005810000034000000001000005
:100A20000705000001030000400000000100000075
:100A30000403000009040000340300004D0000001E
:100A40006900000063000000720000006F000000F9
:100A500063000000680000006900000070000000F2
:100A6000200000005400000065000000630000004A
:100A7000680000006E0000006F0000006C000000C5
:100A80006F000000670000007900000020000000F7
:100A9000490000006E000000630000002E0000000E
:100AA0002603000055000000530000004200000033
:100AB0002000000048000000490000004400000041
:100AC00020000000420000006F0000006F000000E6
:100AD000740000006C0000006F0000006100000066
:100AE00064000000650000007200000006000000C5
:100AF000FF09000001A10000011900000129000008
:100B00004015000000260000FF00000075080000EE
:100B100095400000810000001901000029400000FC
:100B200091000000C0000000EE8400001885000065
:100B30001C850000508500004572000061730000B4
:100B4000696E0000672000004465000076690000BF
:100B5000636500002E2E00002E000000457200008C
:100B60006173000065200000436F00006D7000009D
:100B70006C65000074650000005700007269000099
:100B800074650000204300006F6D0000706C000071
:100B900065740000650A0000507200006573000073
:100BA00073200000526500007365000074000000AF
:100BB000526500007365000074000000754D000070
:100BC0004F470000493200000A4200004F4F00002A
:100BD000544C00004F41000044450000520000000A
:100BE0000080FB008181FB00000140000281410088
:100BF0004311DD0003A020000301410012F0A10019
:100C00000104E00004003A0000004000A180200040
:100C1000823078000300370000004000E1802000AF
:100C20008230780012E0A1006401410012E0A000CF
:100C300000000600214A800080C0B300E78F50000A
:100C40000E003E0001407800818120009140780034
:100C50000104E00004003A0013C0B30082812000C8
:100C60000349780005003700E1CF500003003A0047
:100C700023C0B30082812000034978004194200002
:100C80000081FB00910811007140800080487800CD
:100C9000A1952000D1408800219420009100780087
:100CA000E1806000030032000004E0000C003A0024
:100CB000000006000004E000110032000294200051
:100CC00092017800D140800093587800D14088008C
:100CD0000309E8000040E900F8FF3A0000000600C0
:100CE0000294200092017800D1408000935878004F
:100CF000D14088000309E8000040E900F8FF3A000D
:100D00000000060000C8B30021952000914F10009C
:100D100033003A0001CCB300209420000148780051
:100D20005095200010407800E24F5000090032003A
:100D3000E34F500019003200E14F500026003A0006
:100D4000C04D2800004A880020012000204A880069
:100D500000000600409520001004E0000C003A005E
:100D60001080FB000000400041592800610078001D
:100D7000004A880041942000204190008248780079
:100D80008100E800304090008048780000000600B4
:100D9000209420000048EB00000006004095200051
:100DA00021C0B30090CF100008003E001080FB006F
:100DB000000040006159280061007800004A880066
:100DC0001080FB00204A88000000060020942000CC
:100DD0000048EB0000000600209420000048EB00D3
:100DE000000006000040EB00A1952000804878003C
:100DF0008100E800804878002095200010407800AD
:100E00007F4060000080FB00E10F50000B003200CB
:100E1000E20F50000C0032000000E00028003A0011
:100E2000209420001070A0000348E200240032004B
:100E30000100E9001014A0002100370020942000D8
:100E40001070A0001E003700209420001070A00039
:100E500060952000104078006F406000180032005C
:100E6000609520001004E000070035001040780075
:100E70006F4060000080FB0000004000A180200067
:100E8000E1007800070037006095200010407800EE
:100E90006F4060000080FB0000004000E180200007
:100EA000E10078000040280091006000808F500031
:100EB00003003A0011C0B300A0952000014878005B
:100EC000000820002194200011006000070032007B
:100ED000A0952000004A8800010078001000A000C2
:100EE00021C0B3000080E80001487800000006003F
:100EF000AA24AB0011003200A040800010419000F5
:100F000001C8B300814F51000B003A0071408000CE
:100F10001141900041C8B300814F510006003A00D2
:100F2000C1C0B30011409800A040800090409000E4
:100F30000174A00011409800AA24A9000008200014
:100F40005024880000000600881F78007040800050
:100F5000100478004E44DE00614464000020A200CA
:100F60007040880030408000E80F50000B003A00CD
:100F7000409520001080FB00F007B200B0248800EC
:100F80009604E20003003200000120003040880097
:100F900002003700400020003040880019C8BF0020
:100FA000E14F500021003A00A195200070408000E0
:100FB000110098001FFF070018C8BF00E24F500043
:100FC00008003A0041C0B300704080001140980012
:100FD00070408000904090000174A0001140980083
:100FE000200037000804E00008003A0081C4B30084
:100FF0007040800011409800704080009040900048
:101000000174A000114098001600370081C0B300A1
:101010007040800011409800704080009040900027
:101020000174A000114098000E0037008094200049
:101030001004E0000A003D00514A8000C808DE00AC
:10104000640040001080FB004800DD00008070005C
:101050000100320000000100809420001070A10007
:101060001968EF004F047800000006000468EF00E4
:101070000001EB008200780040072000ED0507002A
:101080008284A90000012000002488000968EF0084
:10109000000006008284A80000012000502488007F
:1010A00010C0B30004E8B7000968EF000001EB00CE
:1010B0008200780050072000DE053700889FBE00C0
:1010C0004095200011C0B30090CF10000E003A00F0
:1010D0000080E900104078007F4060000A003A007C
:1010E000209420001070A0003095200032C0B30082
:1010F000904F110003003A000140780003E8B70068
:10110000010037000368EF00409520001004E00064
:101110009C003A000080E900104078007F406000A9
:10112000E24F500097003A00609520001040780090
:101130006F406000930032006095200010407800FE
:101140006F4060000080FB00E10F50008D003C000C
:10115000000220000608E3008A003A0020942000E4
:101160001070A000609520001004E0000C00350015
:1011700010417800EF4061008180FB0081804000D9
:10118000A280200062847800104078006F406000E8
:101190000080FB0001952000E14478000C0037003E
:1011A0006095200010417800EF4061008180FB00D5
:1011B00081804000E2802000628478001040780046
:1011C0006F4060000080FB00E1942000E144780063
:1011D0000908A30002003A000820A100010037001E
:1011E0000820A000609520001004E00007003500F2
:1011F000104078006F4060000080FB00000040005D
:10120000A18020008830780007003700609520001A
:10121000104078006F4060000080FB00000040003C
:10122000E1802000883078003095200031C0B30084
:1012300090CF10001A003A001800E00013003D00A3
:10124000630040001004E000080035001040780002
:101250006F4060000080FB00019520006141780034
:101260000214A0008270780008003700609520000A
:10127000104078006F4060000080FB00E194200087
:10128000614178000214A0008270780098409000BC
:1012900040C8B30000C07000104498003900370007
:1012A000880078000120A2001100E00008003D0045
:1012B000114090000074A1000064A00090409800CC
:1012C00022002000500020005A05070003003700CC
:1012D000114090000064A000904098000918A300FD
:1012E00002003A001800E0001B003D00609520005D
:1012F0001004E00008003500104078006F406000E6
:101300000080FB0001952000614178000214A100DB
:101310008270780008003700609520001040780047
:101320006F4060000080FB00E19420006141780084
:101330000214A1008270780018409000B043B200FF
:1013400010449800220020008800780050002000FF
:10135000380507000300370018409000B043B20082
:101360001044980060952000104078006F406000A5
:101370000080FB0000004000A14A20000100400066
:101380001014A1004F04BE0000000600881F780062
:10139000209420001070A000AC24EF0008A02000D2
:1013A000020220008000EB00080078007BFD0700AF
:1013B0009424A8000040EB00E194200080487800CD
:1013C0000195200080487800F19420008048780042
:1013D00011952000804878001268EF009424A9003D
:1013E0006800440070408800A8408800B840880029
:1013F000409520001040780008E8B7000004E000A5
:1014000003003A0000012000304088000600370049
:1014100012002000818020000200780005050700EE
:1014200000022000304088004F04780000000600D1
:101430002095200001C6B30010C060003F003A00B4
:10144000309520001080FB008000EB00EB0F500077
:10145000E08F580039003E00006001001C0037009A
:101460001C003700350037001A0037003300370002
:10147000060037000A0037002C0037000A0037004A
:1014800008003700140037002000370020942000A7
:101490001070A0008000200030408800000006008E
:1014A00018FE3700B9FF370080802000004A88000E
:1014B000209420009000780013C0B3000081E80061
:1014C000034978001108B300010878000000060005
:1014D00044FE3700F9FE3700609520001081FB00C4
:1014E0002181200000942000010841000080E800D4
:1014F0009000780013C0B3000081E8000349780031
:101500001108B300010878000000060020942000B4
:101510001070A000609520009080FB0020812000CA
:101520004295200092707800000006000001EB0058
:101530008200780020002000BE04070000000600A2
:101540009EC0A9000080EB00702488005024880011
:10155000AA24EF00AC24EF002000200030258800F2
:10156000A824EF008644A900F00920008024880008
:101570006024880082C4A8008804A80000A020007D
:10158000C800DE00C12488000008EB00301078009D
:101590006000B8002050880031508800405088001A
:1015A0005150880060508800715088008050880039
:1015B00091508800A0508800B1508800C050880029
:1015C000D1508800E0508800F15088009424A80091
:1015D0009624EF0094A4A9009424A9008000200080
:1015E000502488008A64AB00FCFF3A000040EB0006
:1015F0002194200080487800819420000081FB0025
:10160000820878008180E80002F02F0091086100D4
:1016100013C0B30002822000034978001282200028
:10162000034978000268EF000068EF000468EF00EB
:101630000A28EF00E19420008048780001952000FE
:10164000804878001028EF000C28EF00F19420006B
:1016500080487800119520008048780080A0200004
:1016600070408800D0002000502588002095200080
:101670001050880081C0B30000A02000014878000D
:101680000000E80041C0B300014878001074A000D9
:101690000868EF002228EF002428EF000968EF0017
:1016A0000628EF0000000600889FBE008A1F780011
:1016B00000457800814478000984FB000838A300C5
:1016C000030032008040EB000A40780044FD070030
:1016D0000828A3000300320011C0B3000A407800BC
:1016E0003FFD07000A85FB000A054500A04A2000CF
:1016F00009707D004F0578004F04BE000000060011
:101700000104E000050032000082FB0004024200F8
:10171000E580200065027A00040037000082FB00AB
:1017200004024200A580200065027A008002EB00DE
:101730000400E0001A00320012029800034A780008
:10174000144190000244B2001242980014419000EB
:101750000234A00012429800144190000274A000CC
:10176000124298000104E000070032000080FB00F4
:1017700000004000E1802000008040001020A20016
:1017800084027800060037000080FB000000400063
:10179000A1802000008040001020A2008402780078
:1017A00005007800000006000004E00014003A0084
:1017B00081C0B300B040800001487800B040800094
:1017C0002195200011009800C1C0B300114098007D
:1017D000B0408000904090000174A000114098003B
:1017E00041C0B300704080001140980070408000FC
:1017F000904090000174A000114098000000060085
:101800008180FB000080FB00000040000080400061
:101810004300DD0002A0200082014000134290003E
:1018200041C8B30001427200944198006400400036
:10183000020040001041900081407100114098006A
:101840000000060094A4AB00190032000080FB00E9
:1018500000004000E18020000080400090007800FF
:101860001103BE00040420000500200006036200EE
:101870008003EB008688BE00900078001103BE0054
:1018800084186B0085906B00900078000120A20006
:1018900001087800914190000344B2009340980001
:1018A000100078009040900004C168001240980039
:1018B000000006002048E2002A003A0010C0B300F1
:1018C00020E8B7002148E20026003A0021E8B700EE
:1018D00019C8BF00E24F50000A003A007040800073
:1018E0000048EB0081C4B3007040800011409800B4
:1018F00070408000904090000174A000114098005A
:1019000000000600E14F500016003A001E68EF008C
:1019100080C0B300A140800080487800A2408000D1
:10192000219520001101980043C0B3001341980095
:10193000A2408000924190000374A00013419800DF
:1019400014C0B300E381200084497800B2408000D5
:1019500000497800B04080001100980001C8B30031
:101960001140980000000600A0408000104278005E
:10197000414A8000C808DE00A09420001080FB00CF
:101980004800DD00008070008480FB00808F5000E4
:1019900001003600004278008480FB000100500006
:1019A000819420004801DD00F30F20009181610047
:1019B000828871004800DE008180E800804878005D
:1019C0000404E000090032000000EB0061942000F4
:1019D00011017800A3952000634978008208E8008F
:1019E0000000E800804F5200F8FF3E00414A8000AE
:1019F000C808DE00A09420001080FB004800DD0035
:101A0000008070001900320081C0B300B040800037
:101A100001487800A1952000B04080001100980096
:101A2000A040800010E8A30008003A0081C4B30081
:101A3000B040800011409800B0408000904090007D
:101A40000174A000114098000000060081C0B3009E
:101A5000B040800011409800B0408000904090005D
:101A60000174A000114098000000060081C0B3007E
:101A7000B040800001487800B040800021952000EF
:101A80001100980041C0B30011409800B0408000A0
:101A9000904090000174A00011409800514A8000CD
:101AA000C808DE00C09420001080FB004800DD0064
:101AB00000807000010032000000010080942000CE
:101AC0001070A1000148E20001003A0079FF070010
:101AD0000000060019C8BF00E24F500001003A00A4
:101AE000A1FF37001968EF001E48E2000D003A0020
:101AF00081C0B300B040800001487800B040800051
:101B00002195200011009800C1C0B3001140980039
:101B1000B0408000904090000174A00011409800F7
:101B2000000006001E68EF00000006000268EF00DB
:101B30000068EF0019C8BF00E24F50000D003A00E6
:101B400081C0B300B040800001487800B040800000
:101B5000A19520001100980081C4B30011409800A5
:101B6000B0408000904090000174A00011409800A7
:101B700000000600809520001080FB009195200059
:101B80009180FB00C808DD008100700040942000B7
:101B9000908F500007003100809520009080FB005E
:101BA0000000E8001081FB004811DD004094200097
:101BB000010871001FFC0700A19520007040800003
:101BC0001100980081C4B30070408000114098005B
:101BD00070408000904090000174A0001140980077
:101BE0000000060094A4A900000820002194200011
:101BF000110060001F003A00809420001004E000F3
:101C000008003D0020C0B30019E8B7000048E2001A
:101C100001003A00C5FF07002168EF002068EF00CF
:101C20000000060081C0B300B04080000148780089
:101C3000B04080002195200011009800C1C0B30081
:101C400011409800B0408000904090000174A000C6
:101C50001140980041C0B3007040800011409800CE
:101C600070408000904090000174A00011409800E6
:101C700000000600209520001004E0000A003D004E
:101C800010C0B30019E8B7000248E20001003A00B2
:101C9000A6FF07002168EF002068EF000148E2007E
:101CA00014003A0003FF370020C0B30019E8B70062
:101CB00081C0B300B040800001487800B04080008F
:101CC000219520001100980041C0B30011409800F8
:101CD000B0408000904090000174A0001140980036
:101CE0002168EF002068EF000148E20001003A009F
:101CF000F0FE0700000006001868EF000168EF0022
:101D00000268EF000068EF001E68EF001968EF003E
:101D100070408000904090000174A1001140980034
:101D2000704080000020A200704088009040900029
:101D30000174A100114098000E48AA00B040800034
:101D4000904090000174A100114098002094200060
:101D50000048EB008000EB00214A880080942000BE
:101D60008180FB00010878000080E80001F02F006E
:101D700010886000AEFD07000001EB0082007800D3
:101D800030002000AB02070096FF3700D0C2B3003E
:101D90001FE8B700C1812000914078000100780061
:101DA000B00FB20013003A00C10FB20000A0200033
:101DB00080804000A1408800010078000020A2003F
:101DC000B040880002C023001101610000402300E0
:101DD000800F510006003A0011009000219520006C
:101DE00007000900B05878008000B100C2FF37003A
:101DF00038FF3700E80F500001003A0052FC07009E
:101E00000000060010418000214180006100400078
:101E1000E080480010418800214188000448E20029
:101E200004003A000948EC0009E8B70001003A0054
:101E300009E8EF0000000600881F780030408000AD
:101E40000000E00012003A009424EF008C24EF0020
:101E50002000200030258800A824EF008644A90037
:101E6000F0092000802488006024880082C4A80033
:101E70009404AB0003003A009404A8009404AB005F
:101E8000FDFF3200100020003040880002003700C3
:101E9000E10F500008003A0094C4AB0006003A007D
:101EA0008AA4EF008C24EF008C04A8008C84A80086
:101EB00020002000304088008084AB000500320004
:101EC0008284AB000300320000012000002488005F
:101ED00066FC07008824AB00020032008EC0A90017
:101EE000690037008A04AB00070032008C04AB00A5
:101EF0000500320092FD07004000200030408800BD
:101F000010002000502488008A84AB0003003200B7
:101F10008C84AB00010032005EFC070080C4AB0083
:101F2000030032000004200000248800B5FF0700F1
:101F30008A44AB000E0032008C44AB000400320037
:101F4000120020008000EB0030072000390207005B
:101F500040002000502488001FC8BF00030032004A
:101F60000040E9001FE8B70001003A0051FE0700F9
:101F70008AE4AB00030032008CE4AB0001003200C5
:101F8000DBFB07008A24AB00090032008C24AB0085
:101F900007003200120020008000EB00F0FF270055
:101FA000240207008EA4EF002000200050248800A7
:101FB00030408000E30F500002003E008EC0A900B8
:101FC000310037008C64AB002E00320048C0B300F3
:101FD0008A64AB0003003A002A0037008A64AB0031
:101FE0002800320091248000C08120000148780040
:101FF0000181FB004411DE000240780002427800BB
:10200000D381200084497800820020005224880077
:102010000138A30009003A008080FB0002952000EF
:10202000E2C1780061C261000404A2000304A100BF
:1020300084C1710003F17800080037008080FB0044
:10204000E2942000E2C1780061C261000404A200B1
:102050000304A10084C1710003F178000004E000D2
:1020600002003A0049FF0700040037000001EB00BE
:10207000C181200020072000EE0107000844E9008C
:10208000D6FF3A008EC0A9004F0478000000060079
:10209000104180002141800000000600881F780068
:1020A0002628EF002828EF0090CAB3002AE8B700DE
:1020B00000802A00604188002000200070418800D4
:1020C00018C0B30008407800818320008848780059
:1020D0003068EF0034A8EF0036A8EF003268EF0058
:1020E000D1C1B30070FD070003C4B300028C20000F
:1020F0008040EB000840780081FD070030418800F7
:102100004F0478000000060012832000124178007E
:102110000281FB008001EB004A18DD00C610DE00E2
:10212000810070004A10DD0022042400023B880078
:102130008141780022032000034978000081EB00F0
:102140000208BB001000FC0050052000303B880056
:10215000A00A2000303B880061E7A80000000000D2
:10216000000000006007E200FEFF350000000600EE
:1021700030002400003B880032C8BF001D00320040
:10218000019020000081FB008001EB00A441800051
:10219000B54180000201520083815A000342780059
:1021A0002003200004487800020078001108BB00DA
:1021B000110190000288BB001000FC0050052000B7
:1021C000303B8800A00A2000303B880061E7A8006F
:1021D00000000000000000006007E200FEFF350084
:1021E00032C8ED0032E8B700E48040000004E000AF
:1021F000E4FF3A0061C7A9000000060023032000A5
:1022000093417800400ADE00050020000443780076
:102210002203200006497800000178001282BA00EB
:10222000840078001200BA000342780022032000E4
:102230000449780000000600889FBE008A9FBE0007
:102240003048E20022003A00404180000000E000F7
:10225000020032001000E0007301350030418000C0
:102260000000E00005003A00F08B2000F183200020
:102270000204200000014100030037001000E000CC
:10228000F9FF3D0068013700D0687800820F5000E8
:10229000FDFF3A0003C4B300028C20008040EB0035
:1022A00010C0B30016FD07003041880010C0B30015
:1022B00030E8B700F0872000010420008080400053
:1022C0000068EB00810F5000FDFF3A005601370017
:1022D0000084200010407800E54F5000910032004B
:1022E00006003E00E34F50005A0032006E003E00F0
:1022F000E24F50004C013A0006003700E74F500013
:10230000E6003200DB003900E84F500046013A0099
:102310003A01370020C0B3000188200080487800CF
:1023200082C3B3008100E800824878008100E800A1
:102330008048780011C0B300308820000148780040
:102340000040EB00418820008048780082C1B30043
:102350008100E800824878008100E8008048780029
:102360008100E8008048780000802E00F1FF2F00F7
:102370006241800073418000020040008380480079
:10238000F20F200083882000824960004802DE00AE
:102390008301E800844978008301E80082C9600075
:1023A000C808DE000300E800014878000000E800EB
:1023B00000C8EB003848E20019003A0031C0B30011
:1023C000014878000040EB0082CFB300E380410079
:1023D00082487800B2CAB3008100E80082487800E1
:1023E00022C0B3008100E800824878008100E80044
:1023F0008048780082C0B3008100E80082487800FD
:102400008100E800804878008100E800804878007A
:102410008100E800804878000100E80000C8EB0077
:10242000404180000000E000020032001000E000A7
:10243000FD00350003C4B3000288200011C0B300C2
:1024400001407800AEFC0700404188003068EF0092
:10245000F5003700108420001004E00008003A0066
:10246000A0CAB3002AE8B70083BF2A0063418800EE
:1024700023002000734188003868EF00080037000F
:1024800090CAB3002AE8B70000802A0060418800A3
:10249000200020007041880010C0B30038E8B70069
:1024A0003068EF00E00037008000EB0010002000F3
:1024B00010010700C05928005601070060C0B30092
:1024C00031E8B7002AC8BF000080FB000000E80028
:1024D000E60F50000B0034000BFF070056FE07000C
:1024E0003148EC0031E8B7000080FB00A1822000F9
:1024F000914078008180FB008100E800810F50004E
:10250000F5FF350061C7A9003068EF008000EB00DF
:1025100010002000F7000700E05A28003D010700E6
:10252000C1003700A0418000B1418000E10F4000B0
:10253000E08F48000E003A00128420001281FB0058
:10254000238420009381FB00C819DD000300710083
:10255000328420001281FB00438420009381FB0021
:10256000C819DD0083007100A0418800B1418800D6
:10257000128420001281FB00238420009381FB0041
:10258000C819DD0003007100328420001281FB00B5
:10259000438420009381FB00C819DD008300710093
:1025A000A2418000B3418000820F5000838F580009
:1025B0002E003A005084200010407800E14F500077
:1025C0002A0036000044EB0021832000914078006F
:1025D0000181FB00820141000080FB00820320009A
:1025E000000051004F01DE00000041000081D100D9
:1025F0000880FB0000004100640040000000400033
:1026000002842000624278000482FB000000410046
:10261000104190004811DD0002017200009020007E
:1026200002B079000140E80032E8B700A241800022
:10263000B341800061014100E0814900A24188006E
:10264000B3418800FC4F500001003A00C8FE07006B
:102650000844E80050842000104078008080FB008F
:102660008100D100814F5400D7FF39003068EF005E
:102670006D003700BEFE070034A8EF0036A8EF005B
:102680003068EF008000EB00100020009900070088
:10269000D05B2800DF000700630037004041800066
:1026A0000000E000020032001000E0005E00350093
:1026B00071C0B30000882000014878001284200017
:1026C0001281FB00238420009381FB00C819DD00E8
:1026D00003007100328420001281FB00438420003B
:1026E0009381FB00C819DD0083007100F20F200008
:1026F00013882000824960004802DE008301E80060
:10270000844978008301E80082C96000C808DE00BF
:102710000300E80001487800508420001040780051
:102720008380E80080487800E14F50002B0036009D
:102730000044EB000881FB008001EB0014842000C2
:102740001482FB00258420009582FB00C82ADD004E
:1027500005007200348420001482FB0045842000B0
:102760009582FB00C82ADD0085007200020040004F
:1027700083804800A1FE07008884FB005484200069
:102780009482FB008502D1008583FB0007855400FD
:102790000A02B000068820000A0545000A05430029
:1027A000F40F2000044D6000C805DE001B459800B2
:1027B00081016200078054001002B0000000400058
:1027C0000000430004C86100C818DE0011409800F2
:1027D00008C4E80088CF5200D6FF3E0003C4B3000F
:1027E0000288200011C0B30001407800C4FB07003C
:1027F000404188003068EF000B0037008000EB009C
:10280000100020003B000700805D280081000700C9
:102810009424EF000080EB00000000000000E900BD
:10282000FDFF3A000000FE004F05BE004F04BE0051
:102830000000060031072000810F50000D0032001B
:1028400005003C00E10F500010003200E30F500083
:1028500011003A000F00370041072000810F50009F
:10286000080032008100E800810F50000A003A00A1
:1028700002003700FE00070007003700FC000700D9
:1028800005003700FA0007000300370003FE0700C9
:10289000010037007100070010000500EC22A800BD
:1028A000000000000000000000000000EC22A90071
:1028B0000000060000F02F00E022B600F002A900A0
:1028C000F022A900E822A900F402A900F422A9003C
:1028D000EC22A900000006000000FB0001F02F0020
:1028E000221780008280600080807000211788009D
:1028F0000000060080417800F00F2000E022B700C1
:10290000F422A800F402A900EC22A80000000000B4
:10291000000000000000000012178000EC22A90057
:102920000278A300F8FF3A0002F02F00002E2000EA
:1029300010086100F422A9008180FB008100EA00F8
:10294000CF08DE00A21780000200A1000281700003
:10295000A217880003407800DFFF0700CFFF370091
:10296000D4FF070000202100A10720001801070064
:102970008040EB0080C3B300DEFF07008040EB0027
:1029800080C0B300DBFF07008040EB0010C0B30045
:10299000D8FF07008040EB0060C0B300D5FF070000
:1029A0008040EB00C0C0B300D2FF070000B82B008E
:1029B0000100200006013700F0F32F004427B60085
:1029C00042A7AB0003003A000000000042A7AB00A2
:1029D000FDFF320040A7A900F0C2A900D022A80044
:1029E000DFFF07000000EB00E3000700D4FA070058
:1029F0000060FE0010FD070030408000FF0F500017
:102A0000FBFF36008824AB00F9FF3A000AFE0700FE
:102A1000F7FF3700881F780000047800184078001E
:102A20000004E0000B003200EA4F500004003A00BE
:102A30008040EB0000CCB300AEFF0700020037007F
:102A400011C0B300ABFF0700584078000004E0005D
:102A5000F5FF3A004F0478000000060020952000A2
:102A6000104078007F406000E14F500054003A0071
:102A7000609520001004E00051003A00630050000F
:102A800061C0B30090CF10001B003A000080E80046
:102A900010407800FBC04000814F5000040032001D
:102AA0008140E800814F500013003A000B003700CE
:102AB00008C8BF00E14F50000F003A000050280046
:102AC000004A880090002000204A880001CCB30012
:102AD0002094200001487800070037006057280044
:102AE000004A8800D0012000204A880001CCB300B1
:102AF00020942000014878002095200002C6B300F1
:102B00009040610000C2B30080CF50002C003A001A
:102B10003095200010407800E34F5000190032003B
:102B200003003E00E24F500025003A000500370048
:102B3000EA4F50000B003200EB4F500020003A00EB
:102B400018003700A0832000004A880010002000F1
:102B5000204A880011CCB30020942000014878005E
:102B60000000060001C8B30020942000014878004E
:102B70005095200010417800A18320008248780001
:102B800000000600B0832000004A880010002000EA
:102B9000204A880011C8B300209420000148780022
:102BA0000000060001C8B30020942000014878000E
:102BB0004095200010417800B183200082487800C1
:102BC00000000600E10F500003003200E20F500049
:102BD00004003A0002003700F4C2A800000006001A
:102BE000F4E2A80000000600E10F500003003200EC
:102BF000E20F500004003A0002003700F4C2A900BE
:102C000000000600F4E2A90000000600E10F5000F9
:102C100003003200E20F50000B003A0005003700BD
:102C200000042000F402B6000000EA004F00DE00BD
:102C30000000060000082000F402B6000000EA00D0
:102C40004F00DE000000060000000500E10F50000C
:102C500003003200E20F500004003A000200370087
:102C6000F0C2A90000000600F0E2A9000000060082
:102C70008824AB000200320010002000DAFF370089
:102C8000000220000608E30010003A00F041800036
:102C9000E10F500002003A00CAFF07001A00370097
:102CA000B1042000810F500003003A001000200002
:102CB000CDFF07001400370061092000810F50008C
:102CC000110036003E28EF000F003700F041800071
:102CD000E10F500002003A00BAFF07000A00370077
:102CE00021032000810F500003003A001000200053
:102CF000BDFF070004003700613B2000810F50003A
:102D0000010036003E28EF003E28EC0000000600DF
:102D10004009000022000000000000000008000040
:102D20002600000000000000000A00002000000053
:102D3000000000003A08000002000000000000004F
:102D4000400800000001000000000000260800000C
:102D500014000000000000003C0800000200000019
:102D600002000000010000003E0800000200000018
:102D700000000000000000000000E00013003A0026
:102D800083E0A800100020002700070010002000AA
:102D90001D0007000004E00006003A003008200093
:102DA0004007B6000300320083E0A900001A0400C7
:102DB00000000000E05D280016FF07001000200062
:102DC000A2FF070020002000A0FF0700000006006F
:102DD000F03FB1000180B10006003500EE030900AC
:102DE00000000000403FB1000180B100FBFF3D004A
:102DF0001000B000203FB000020035000080090044
:102E00000000000000000600E10F500005003A003D
:102E100090168000620060000000E9004F00DE00B4
:102E20000000060000000500E10F500001003A001C
:102E3000D022A80000000600FFFFFF00FFFFFF00F8
:10340000101B040000000000001C0400000000006D
:10341000001C040000000000001C0400000000006C
:10342000001C040000000000001C0400000000005C
:10343000001C040000000000001C0400000000004C
:10344000001C040000000000001C0400000000003C
:10345000001C040000000000001C0400000000002C
:10346000001C040000000000001C0400000000001C
:10347000001C040000000000001C0400000000000C
:10348000001C040000000000001C040000000000FC
:10349000001C040000000000001C040000000000EC
:1034A000001C040000000000001C040000000000DC
:1034B000001C040000000000001C040000000000CC
:1034C000001C040000000000001C040000000000BC
:1034D000001C040000000000001C040000000000AC
:1034E000001C040000000000001C0400000000009C
:1034F000001C040000000000001C0400000000008C
:10350000001C040000000000001C0400000000007B
:10351000001C040000000000001C0400000000006B
:10352000001C040000000000001C0400000000005B
:10353000001C040000000000001C0400000000004B
:10354000001C040000000000001C0400000000003B
:10355000001C040000000000001C0400000000002B
:10356000001C040000000000001C0400000000001B
:10357000001C040000000000001C0400000000000B
:10358000001C040000000000001C040000000000FB
:10359000001C040000000000001C040000000000EB
:1035A000001C040000000000001C040000000000DB
:1035B000001C040000000000001C040000000000CB
:1035C000001C040000000000001C040000000000BB
:1035D000001C040000000000DC1B040000000000D0
:1035E000001C040000000000001C0400000000009B
:1035F000001C040000000000001C0400000000008B
:10360000001C040000000000001C0400000000007A
:10361000001C040000000000001C0400000000006A
:103620000FC220000E7F24000E0188000000000061
:10363000000020000000E000020032000001200035
:103640002002880014000700B10007000000E0001D
:1036500003003A00A06E24000100200002003700A1
:103660000000200001002000810F700001003200E6
:1036700014000700000020000000E00002003200FB
:103680000000020000000000DA4802000000000014
:103690000040DA000000FE004440A90000102000B5
:1036A0000000E0000300320000002000A0018800BC
:1036B0004440A800000006008A1F78008B1F780095
:1036C0000000060091018800800478000000EB00F3
:1036D0001A003700E284440032A0B4009905BA0011
:1036E000E284440032A0B4009906BA00E2844400A7
:1036F00032A0B4000006EB00476FDE00FD07B20009
:10370000636CE10003003A00EBFF07000000EB00F0
:103710000A003700606CE10004003A00005DEB0035
:103720008B05E900FDFF3E00040037006168E10001
:10373000010032000086EB000B00070019C7BA0039
:103740001905BA000E04E00003003A000A00E00088
:10375000E0FF3A0000000600FE07B2009E0188006C
:103760008A047800F5FF3700395DBA008B05E9005F
:103770000C003200295DBA008B05E9000800320018
:103780000C00E00003003A00E284440032A0B400E0
:10379000F5FF370019DDBA008B05E900FAFF3A00A2
:1037A0008904E800E184440032A0B400000006006F
:1037B00094410400000000003600F800809FBE0025
:1037C000829FBE00849FBE00869FBE003400F8002A
:1037D00000002000A00188000000FA00FF09070097
:1037E0000080FA003400F9004F03BE004F02BE0013
:1037F0004F01BE004F00BE003600F9000040060039
:103800000040DA000000FE000A00FA00E20F50005B
:1038100034003E0080528000E10F5000030032006F
:10382000E20F500011003A000C0037000322200084
:103830000300E00001003A000040DA002002E2004C
:10384000020035002822EF0021E2A8002342AB004D
:103850000D003A002342A8000B003700032320008C
:103860000300E00001003A000040DA003002E2000C
:10387000020035003822EF0031E2A8003342AB00ED
:1038800001003A003342A800820178000B003700A3
:103890003102FB00E10F500004003A002322AB008C
:1038A000FEFF3A0024118800030037003322AB00EA
:1038B000FEFF3A00A41188008301E9000300E00044
:1038C000F3FF3A00E10F500003003A002302AB007F
:1038D000FEFF32000B0037003302AB00FEFF320068
:1038E0000800370033002000B3BF9F00C0BF9F0017
:1038F000D1BF9F00E2BF9F006A8057008807070082
:103900006FB99700020078000080FA0000000600FE
:10391000000005002800FA00889FBE008A9FBE00B4
:103920008C9FBE0003866B00800007006400E100EE
:10393000440032006408E1004A0032006100E10006
:10394000460032006108E10049003200EC06470001
:103950006000B8003D02BE003D03BE00F486570083
:103960006011B8003D04BE003D05BE007D0320008F
:103970000B0037000000A0008D06E90013003200A4
:103980000402420085824A0006034B0087834B00F5
:103990000000400081804800020149008381490005
:1039A0000802520089825A000A035B008B835B0085
:1039B000F0FF3B000802420089824A000A034B00E4
:1039C0008B834B008D06E900EDFF3A008482720084
:1039D00086827200F707B20087827200010032000F
:1039E000150020001E0490003E0B900006035400BA
:1039F000E63FB0000368A300070032000000A70004
:103A00000500A0008301D1000281D3008180D30092
:103A10000080D3000603E8008301D1000281D300B7
:103A20008180D3000080D3000002EB000482D2002A
:103A30001200070003F0A1000CF0A70003F0A000A3
:103A40004E003700640247006408E100480032007D
:103A50003400BE003401BE00F6FF37006108E1000B
:103A6000430032006011B8006000B800F1FF370079
:103A700003FF270002002000FBFF37001800200092
:103A800057002000080453000D003D0006002000F0
:103A900097FC2F000740E1001E0034008482720072
:103AA000610260008301D1000281D3008180D300D4
:103AB0000080D3000804E800F8FF3A004700200027
:103AC0006104600005047400040464000D00320009
:103AD00061004000E080480060014900E081490049
:103AE00003B8A500070032000603E8006538E100CE
:103AF00004003A008301D1000281D3008180D30009
:103B00000080D300F87F20000830E100030035007A
:103B1000080378006000B8006011B8004433DD008D
:103B2000F300B20083017300000006006804470040
:103B30000294BE000094BE00FC0447008694BE00C0
:103B40008494BE00090078009900070008007800FE
:103B50009700070099007800814F70000B003B0030
:103B60000800BE00840007004F00B10003003700CA
:103B7000F3FF2700F2FF2F006110B9004F06BE00CF
:103B80004F05BE004F04BE000080FA000000060092
:103B90004F89DE0082017800AC0037000000000091
:103BA0002800FA00889FBE008A9FBE008C9FBE003E
:103BB00003866B00DDFF07000028A30064003A00C5
:103BC0000128A30067003A000008A30062003A0041
:103BD0000108A30065003A001E009000BE08900096
:103BE00081064000ED3FB100F4805700EE019000E7
:103BF000111AB8008E099000311BB8009E09900080
:103C0000311CB800511DB800F4855700460007006C
:103C1000FE0190003A0007008B85E8003E00070097
:103C20008E09900040000700EE019000340007006C
:103C30008B85E800380007008E09900040000700DF
:103C40009E0990001B18B800890440000A854800AE
:103C5000FE019000340007008B85E8003800070063
:103C6000EE019000300007008E0990001B18B8008C
:103C7000890440000A8548000A98A30008003A0019
:103C80000402420085824A0006034B0087834B00F2
:103C900008044C0089844C000A054D008D06E9009B
:103CA00084827200850273004C3ADD008502720046
:103CB0000100320015002000443ADE001400B2007A
:103CC0004538DE00CB45DD000B007000C540DE004E
:103CD000CB4DDD008B8070004549DE00CB55DD000B
:103CE0000B017100C551DE000D03780063FF070072
:103CF00003F0A1000CF0A70003F0A0009FFF370025
:103D00001B18B8008502400006834800E0834B0082
:103D100060044C00070037001B18B8000603400081
:103D200087834800FAFF37001B18B800870340005C
:103D300008844800E0844C0060054D000000060047
:103D40001B18B8000804400089844800FAFF3700B7
:103D50000108A30086FF3A005800BE005801BE00CB
:103D6000E3FF37000008A30081FF3A000904780050
:103D7000F9FF370000000000E48240001078A30043
:103D800007003200640240001178A3003400BE0036
:103D90001401BE00040032000330A700000006003A
:103DA0003500BE001501BE000330A0000000060073
:103DB000800078005002BE005003BE004439DE008F
:103DC000F700B200F37F2000030161000900320018
:103DD0000218E10016003A008501720083017300A9
:103DE000838173000008200015003A004000200085
:103DF0001300370085017200830173008381730013
:103E000005003A0004A8BE0006A8BE00100020006D
:103E10000B0037000201E9000402420085824A00DB
:103E200006034B0087834B000748A300F9FF3200CD
:103E30000740A00004A8BE0006A8BE002000200085
:103E4000800098009200980000000600881F78000B
:103E5000030478000300E00007003D00600010004C
:103E6000E080180060011900E081190002003B00A9
:103E700001F02D00030037000400070008F0A70040
:103E800003F0A0004F04780000000600889FBE00E9
:103E9000008270000402710004827100240032006C
:103EA00036432000C50020008383CF000A0039007C
:103EB0000541B1008283CF00070039000541B10000
:103EC0008183CF00040039000541B1008083CF0019
:103ED000010039000541B10085C353006022B800DC
:103EE000120032000A003B0084827200610260000E
:103EF0008301D1000281D3008180D3000080D300F0
:103F00000603E8008743E800F7FF3A0007003700A0
:103F1000000040008180480002014900838149007F
:103F20000603E9008743E900F9FF3A00D3FE0700E2
:103F30004F04BE0000000600800178000200370038
:103F4000B15978000201E9000200E000FCFF3A00EC
:103F500000000600800178000200370081597800D7
:103F60000201E9000200E000FCFF3A000000060048
:103F70000C00FA00889FBE0000047800F0FF2700C4
:103F8000D0BF9F008004EB0099BF9F0088BF9F00B7
:103F9000A8BF9F00200C2000B0BF9F007881570071
:103FA000CFB0970070805700D00007000FB897007F
:103FB000094878008FB89700088050004F04BE0071
:103FC0000080FA00000006000800FA00889FBE008A
:103FD0008A9FBE000084FB00D1C6B300814F500011
:103FE000340036004B062000110009000B84D80075
:103FF00081057800720040004300DD00E98E20005A
:10400000008044006022B8000600200007FE230064
:104010005001BE004000BE00E1FE07000002BE00ED
:104020000203BE0084BF9F0095BF9F00A6BF9F00F4
:10403000B7BF9F00AA002000110009008A85D800A0
:1040400080057800E9854500C35DDD008B8544006F
:104050003B02BE002B03BE000FB897009FB897002D
:104060002FB99700BFB99700CDFE07000002BE0030
:104070000203BE0084BF9F0095BF9F00A6BF9F00A4
:10408000B7BF9F00110009000A84D800010478001E
:104090004344DD00888444003902BE002903BE0089
:1040A0000FB897009FB897002FB99700BFB9970036
:1040B0001D003700EA4F500013003600AA00200010
:1040C000110009000A84D800010578006904400045
:1040D0004344DD00E98E2000088444006022B800DB
:1040E0000600200007FE23003800BE002801BE00A5
:1040F000ABFE07004355DD008A8444003902BE0050
:104100002903BE00080037004344DD00E08E200094
:10411000080440006022B8000600200007FE2300CB
:104120003800BE002801BE009DFE07004F05BE00FE
:104130004F04BE000080FA00000006000800FA00EC
:10414000889FBE008A1F780000047800D0062000F7
:104150000800E0001F003D000804EA00800F540042
:104160000700340042062000110009000204D800B4
:10417000720040004300DD00E98E20001D00370082
:10418000EA0F540010003400A200200011000900C2
:104190000204D80001047800690040004300DD00FB
:1041A000E18E2000008040004344DD008880400014
:1041B0003102BE002103BE005001BE004000BE001F
:1041C00077FE07003C0037004344DD00E08E20000E
:1041D00036003700800F54002500340042062000CE
:1041E000110009000204D800720040004300DD0005
:1041F000E983200080814400AA002000110009000A
:104200008A00D8008000FD00E9804000C308DD007E
:10421000818044003102BE002103BE003300BE0095
:104220001301BE005EFE07000002BE000203BE00D6
:1042300094BF9F00A5BF9F00B6BF9F00C7BF9F0050
:10424000110009000A04D800010478004344DD008D
:10425000888444003902BE002903BE001FB89700BD
:10426000AFB897003FB99700CFB99700D4FF370098
:10427000EA0F54000B003400A200200011000900D6
:104280000204D80001017800690040004300DD000D
:10429000E1832000008040004311DD008280400067
:1042A000C3FF37004344DD00E083200008044000E2
:1042B0003800BE002801BE004F0578004F04BE0044
:1042C0000080FA0000000600D00190000281510039
:1042D0004240A90003003400100178000149780031
:1042E0000208E80001007800000006006F02B0003C
:1042F000889FBE008A9FBE008C9FBE008E1F7800E4
:1043000000067800B1AF9F0082B79F006000B80040
:104310006011B800C0AF9F00D1AF9F00E2AF9F0017
:10432000F3AF9F008006EB006F043700BFA8970033
:104330008100E800B1AF9F0051C2B300814F50002F
:1043400003003A00BFA997000000EB0011003700FE
:10435000BC0090000000FB000168A30007003200D1
:104360000D017800800078000C007800D6FF07006F
:104370000000E00005003A005B0437008C00780084
:1043800065040700E10F4000570432008D06E80085
:104390005504370003017800B3407800D4C2B3005D
:1043A00084CF50000C00320007003C006D425200E8
:1043B00084CF50000A0032006B42420084CF50008C
:1043C0000D003A000800370004C3B30084CF50004A
:1043D00009003A00060037000030A000EDFF37006A
:1043E0000000A000EBFF37000010A000E9FF37003D
:1043F0000020A000E7FF37000018A30001003200F2
:104400000000A1000038A300010032000020A1003C
:104410008101FB000303B100E98F51000C003E0055
:10442000820178008005EB006A5AB900B305FB00F1
:104430000B03B10084854500030178009300FB0065
:104440000103B100E98F5000F7FF36000800370084
:104450008005EB00A3C2B30083CF500004003A00F4
:104460008FB19700C305780083B79F000201E80071
:10447000E1C2B30092CF100017003A0000E0A000A4
:10448000E4C05000D2CF1000040032008200780057
:104490000002EB00E4B79F00080037008FB29700DE
:1044A0004503780085B79F00E6B79F000201E8004A
:1044B0000C0037006A22B900048241000101780033
:1044C000B101FB000303B100E98F5100F9FF360091
:1044D000E4B79F000300370000C0A0008003EB009A
:1044E000E7B79F00B2407800B2AF9F00C3C6B300E9
:1044F00083CF50001400320009003C0032C6B300E4
:1045000082CF5000790032006341410082CF5000D9
:104510000F0032000104E000F80332008C00370085
:1045200052C7B30082CF50008E0032006341410079
:1045300082CF5000090032006541510082CF500007
:1045400083003A00080037000040A000E5FF370074
:10455000E1CF9F0000A0A00084003700E1CF9F00C2
:104560000070A00081003700E1CF9F000FB29700DC
:10457000C400780084B79F00010478000100E000C7
:1045800001003A00E8992000080178008000EB0063
:10459000010037008100E800E2C178000304E00078
:1045A000FCFF3A0081047800EFB297000500E000BC
:1045B00003003200898F5200010031008504780029
:1045C0000005EB00898F5500010036000985550074
:1045D000E80560002A003A00110037003C00900016
:1045E0000068A300070032000D01780001022000DE
:1045F0000C00780034FF07000000E00006003A00DD
:10460000060037008C00780000022000C20307007B
:10461000E10F4000010032008D06E8000A05E900C4
:104620000A00E000EDFF3A000085EB0014003700BF
:104630003C0090000068A3000900320008007800E8
:10464000B000FB00000478000D0178000C00780039
:104650001DFF07000000E00008003A0008003700D6
:10466000880078003100FB00010478008C0078009D
:10467000A9030700E10F4000010032008D06E800A9
:10468000090078008004E9000000E000E8FF3A003B
:104690000B00E00094033200110037003C00900052
:1046A0000068A300070032000D017800010220001D
:1046B0000C00780004FF07000000E00006003A004C
:1046C000060037008C0078000002200092030700EB
:1046D000E10F4000010032008D06E8000A05E90004
:1046E0000A00E000EDFF3A007F0337000FB39700A8
:1046F0004602780086B79F00CFA2DE00C82BDD00FF
:104700004821DE0002817300C829DE00E2CF9F004D
:104710000048A300080032000204E0000600320056
:10472000E14F410004003200F2CF9F0084D79F0088
:104730002900200002003700F4CF9F00190020005C
:10474000E1FC2F008F8040000104E80096FF370055
:10475000E1CF9F00E8FC2F000F0444001900200067
:1047600091FF3700E1CF9F00000CB300D0B79F004E
:10477000007020005FB1970000006100F00161004F
:10478000A3AF9F000000E0002502320002C8A30092
:104790000200320064002000E4B79F008FB297004F
:1047A000688052002FAB97000600E000090032003D
:1047B00080B79F00800078005101BE004100BE001C
:1047C00090B79F00A1B79F00B2B79F00C3B79F00EB
:1047D0000800370080B79F00800278005503BE00B4
:1047E0004502BE0094B79F00A5B79F00B6B79F00D3
:1047F000C7B79F006022B8006033B8001FB09700B1
:10480000AFB097003FB19700CFB1970044040700C5
:104810000000E0000C003D001FB09700AFB0970013
:104820003FB19700CFB1970003F0A20090B79F006F
:10483000A1B79F00B2B79F00C3B79F00DFB097003A
:104840003100B300D1B79F000000EB0090AF9F0094
:104850006022B8006033B8001FB09700AFB0970077
:104860003FB19700CFB19700370407000000E00088
:104870003400320024FD2F000F0242001FB09700C9
:10488000AFB097003FB19700CFB197006604070023
:104890001FA897000000E9006302B900A2002000F1
:1048A000110009000202D80090AF9F000000E00054
:1048B00002003D000000E90090AF9F001FAC970090
:1048C0000800EA001DFE07001FB29700AFB2970074
:1048D0003FB39700CFB39700B1FC07000002BE00C2
:1048E0000203BE00C4AF9F00D5AF9F00E6AF9F009C
:1048F000F7AF9F006022B8000600200007FF2300EA
:10490000070407000000E00002003D000804E90081
:104910000B0037006022B800060020004702240088
:104920004FA89700DFA897006FA99700FFA99700ED
:10493000000407000000E000020035000804E80061
:1049400098AF9F00EFB29700EC8F52000F003C0031
:10495000054078009CFD07000002BE000203BE0077
:104960001FB09700AFB097003FB19700CFB197004D
:104970006D0307000002BE000203BE0094B79F0053
:10498000A5B79F00B6B79F00C7B79F001FAC9700A1
:10499000E90F540015003C006022B8006033B800F5
:1049A0001FB09700AFB097003FB19700CFB197000D
:1049B000E50307000000E000310032001FB097005F
:1049C000AFB097003FB19700CFB19700E303070066
:1049D000E00F5000E08F5800E00F5900E08F5900C1
:1049E00027003A00E10F54002500340054692D00DF
:1049F00065822E00B6E02200170124004FA8970020
:104A0000DFA897006FA99700FFA99700C4030700CC
:104A10000000E00002003D0069045400010037007E
:104A20006804540098AF9F001FA89700C3FD0700BB
:104A30000002BE000203BE00C4AF9F00D5AF9F00BE
:104A4000E6AF9F00F7AF9F001FB09700AFB0970091
:104A50003FB19700CFB19700AEFB0700BF0307003F
:104A60000004BE006000B8006011B80090B79F005D
:104A7000A1B79F00B2B79F00C3B79F0016003700D1
:104A80001FB09700AFB097003FB19700CFB197002C
:104A9000B20307000004BE00E10307000002BE00ED
:104AA0000203BE001FB09700AFB097003FB1970060
:104AB000CFB19700F90307000002BE000203BE0059
:104AC00094B79F00A5B79F00B6B79F00C7B79F00D8
:104AD0000000EB0090AF9F00619B200010C0B3006E
:104AE00005003700E4804000B10F5400A18F5C0046
:104AF000030039000040E800EA4F5000F9FF3A0097
:104B0000E0CF9F009FA8970081805500EFB29700EB
:104B1000858050000000FB00008550000500E0008B
:104B2000010032000A05E9005FB3970063006300EB
:104B3000010032000A05E900DFB397000728A3004F
:104B400039003200618163000718A3000F003200B2
:104B50003C0090000068A30006003200B102200073
:104B60000200E000010032008180E8000D017800C1
:104B70000D003700B00220000200E000010032000A
:104B80000080E8008C0078000E0037000200E00092
:104B9000220032003C0090000068A30007003200B1
:104BA0000D017800010220000C007800C6FD07000E
:104BB0000000E00006003A00180037008C00780082
:104BC0000002200054020700E10F400013003200F1
:104BD0008D06E800110037003C0090000068A3003B
:104BE000070032000D017800010320000C0078005E
:104BF000B5FD07000000E00006003A00060037009F
:104C00008C0078000003200043020700E10F400001
:104C1000010032008D06E8000A05E9000A00E00004
:104C2000EDFF3C00590037005FB097000038A3004B
:104C300014003A00110037003C0090000068A30007
:104C4000070032000D017800010220000C007800FE
:104C50009DFD07000000E00006003A000600370056
:104C60008C007800000220002B020700E10F4000BA
:104C7000010032008D06E8000A05E9000A00E000A4
:104C8000EDFF3C00DFB09700618160000118A300D8
:104C90000E0032003C0090000068A30005003200C6
:104CA000B10220000200E000220032008180E80012
:104CB00020003700B00220000200E00001003200B6
:104CC0000080E8008C0078002C0037000200E00033
:104CD0002E0032003C0090000068A3000300320068
:104CE0000D01780001022000130037008C007800CD
:104CF00000022000210037003C019000619B200051
:104D00000000FB000268A300100032004200DD003A
:104D1000008040001001BE000800BE0061030700D3
:104D2000A2002000030020006E0307000103200002
:104D3000808040000D0178000C00780062FD0700C3
:104D40000000E00010003A00100037004200DD00D3
:104D5000008040001001BE000800BE0051030700A3
:104D6000A2002000030020005E03070002032000D1
:104D7000000141008C00780002007800E601070085
:104D8000E10F4000010032008D06E800EFC89700F7
:104D90000140E900E0CF9F000104E000D6FF3A00A7
:104DA000130037003C0090000068A30007003200A9
:104DB0000D017800010320000C00780042FD07007F
:104DC0000000E00006003A00060037008C00780082
:104DD00000032000D0010700E10F40000100320075
:104DE0008D06E8001FA897000000E90090AF9F0023
:104DF0001FA897000000E000EAFF3C006FB1970099
:104E0000E80F51000300340080C0B300E0CF9F00E2
:104E100002003700CFE99700E3CF9F006FC89700EB
:104E20008005FB006FB297008B0552000004E00084
:104E3000100032003C0090000068A3000700320020
:104E40000D017800E10220000C0078001EFD070033
:104E50000000E00006003A00060037008C007800F1
:104E6000E0022000AC010700E10F40000100320029
:104E70008D06E800EFCA97000500FB00AFFC0700B5
:104E80000002BE000203BE001FB09700AFB0970043
:104E90003FB19700CFB1970041FB0700AF02070079
:104EA0002D0037003C019000619B20000000FB00BA
:104EB0000268A300100032004200DD008080400044
:104EC0001101BE000800BE00F6020700A20020008B
:104ED000030020000303070001032000808040003E
:104EE0000D0178000C007800F7FC07000000E000DE
:104EF00010003A00100037004200DD0080804000C2
:104F00001101BE000800BE00E6020700A20020005A
:104F100003002000F302070002032000000141000B
:104F20008C007800020078007B010700E10F400050
:104F3000010032008D06E8006FCB97000600FB00F1
:104F40004200DD00619B2000008040001001BE0097
:104F50000800BE00E30207000004BE00EFC897008F
:104F60000140E900E0CF9F000104E000CDFF3A00DE
:104F7000110037003C0090000068A30007003200D9
:104F80000D017800010320000C007800CEFC070022
:104F90000000E00006003A00060037008C007800B0
:104FA000000320005C010700E10F40000100320017
:104FB0008D06E8008B05E9000B00E000EDFF3A00EC
:104FC000DFB397000738A300470132000A00E00072
:104FD000450134003C0090000068A3000700320047
:104FE0000D017800010220000C007800B6FC0700DB
:104FF0000000E00006003A00060037008C00780050
:105000000002200044010700E10F400001003200CF
:105010008D06E8000A05E900EEFF3A00320137008C
:105020002FA897000000E000040032008FB0970026
:105030004104BE0081B79F00040037000FB1970004
:105040004204780082B79F008004EB00EFB1970024
:105050000300E00006003A000880740000F0A7009A
:105060000000EA000000E9004F00DE00E0B79F000A
:105070005FB29700040CB20094B79F0000082000B4
:10508000800F52000D003200000C2000800F5200F3
:1050900018003A00619B200010C0B300E48040007B
:1050A000B10F5400A18F5C00110039000040E800EE
:1050B000EA4F5000F9FF3A000D00370010C0B3006E
:1050C0000201200003002000820F5400838F5C0047
:1050D00007003900C41ADD00CC11DE0083817200A4
:1050E0004411DD000040E800E84F5000F6FF3A00B0
:1050F000E0CF9F006FCB97000600FB00EFB3970057
:10510000870F500002003D00E7CF9F0004003700EA
:10511000EFB09700808F500001003D00E0B79F0086
:105120000B00E000040032005FB1970063006100F3
:10513000010032008B05E900DFB1970003E8A3000E
:10514000060032006FB29700848F550002003400D1
:1051500084855500010037008005EB00EFCA9700F9
:105160000500FB000007EB00808F550001003400B4
:10517000008755005FB397000628A300380032006F
:10518000610163000618A3000F0032003C0090008C
:105190000068A30006003200B10220000200E00017
:1051A000010032008180E8000D0178000D00370019
:1051B000B00220000200E000010032000080E800A0
:1051C0008C0078000E0037000200E0001000320072
:1051D0003C0090000068A300070032000D01780039
:1051E000010220000C00780037FC07000000E000FE
:1051F00006003A00060037008C007800000220000C
:10520000C5000700E10F4000010032008D06E800F4
:105210000E00E0004E0032003C0090000068A30049
:10522000070032000D017800010320000C00780017
:1052300025FC07000000E00006003A0006003700E9
:105240008C00780000032000B3000700E10F40004D
:10525000010032008D06E8000E07E900ECFF370080
:105260000E00E00015003200DFB397000738A300FE
:1052700012003A003C0090000068A30007003200D2
:105280000D017800010220000C0078000EFC0700E0
:105290000000E00006003A00060037008C007800AD
:1052A000000220009C000700E10F400001003200D6
:1052B0008D06E8000E07E900EEFF3A005FB09700A8
:1052C000610160000018A3000F0032003C00900054
:1052D0000068A30006003200B10220000200E000D6
:1052E000010032008180E8000D0178000D003700D8
:1052F000B00220000200E000010032000080E8005F
:105300008C0078000E0037000200E0001000320030
:105310003C0090000068A300070032000D017800F7
:10532000010220000C007800E7FB07000000E0000D
:1053300006003A00060037008C00780000022000CA
:1053400075000700E10F4000010032008D06E80003
:10535000EFB097000102E9004222DD00609B2000CF
:1053600000024200810578000405780045003700FE
:105370008B05E900000820001FB19700800F510045
:1053800021003200000C2000800F51002B003A0059
:10539000AFA997000300E000100032001A02BE001F
:1053A0000401BE000800BE00F4B79F0085BF9F0047
:1053B000BC010700E0CF9F000000FB00CF80DE00B3
:1053C0007FB297008FBA97000401BE00C8010700A2
:1053D0000004540081845C00070037001A01780043
:1053E000110009000284D800A20020001100090069
:1053F0000280D800E1CF9F006FCA97000443B0003D
:10540000E4CF9F000D003700609B20000000550096
:105410000803BE00000178000201E9000300330028
:105420008703D1000683D300FBFF37006F006300C2
:10543000519A200061407800E0CF9F00BC009000AE
:10544000EFC997000300FB000168A30007003200CA
:105450000D017800800078000C0078009AFB0700AE
:105460000000E00005003A00050037008C007800DD
:1054700029000700E10F4000010032008D06E8001E
:10548000640555000B00E000B9FF3A005FB29700D9
:105490000438A300140032000E00E00012003400B3
:1054A0003C0090000068A300070032000D01780066
:1054B000010220000C00780083FB07000000E000E0
:1054C00006003A00060037008C0078000002200039
:1054D00011000700E10F4000010032008D06E800D6
:1054E0000E07E900EEFF3A00BFAA970015407800CA
:1054F000E0CF9F000004E0008CFB3A000D00780034
:105500004F0778004F06BE004F05BE004F04BE0097
:105510006F02B10000000600889FBE000104780001
:10552000B80090008084EB000118A3003A0032001C
:10553000180190000198A30002003A000200E00068
:1055400035003A000190A0003104980080047800F2
:10555000F90FB2000200E00002003A0028009000BB
:10556000000C7800EA8F540005003A000178A3008F
:1055700003003A0088007800D0002000E6FF070012
:1055800018009000D8009000810F50000B003200EE
:105590000000E8001004980018007800094878001E
:1055A000000CE80011C0B300A0A42000014878005E
:1055B000EA8F540018003A00050037008800780090
:1055C00009407800170007008004780012003700B7
:1055D000380090000088A3000F00320018019000EE
:1055E000A80090004800900087F8070098009000FD
:1055F000810F500004003200380090000003B30017
:10560000300498008084EB000000EB001004980048
:1056100028009000000C7800090078004F04BE00BC
:10562000000006000200FA00889FBE00A0FF9F0055
:1056300001047800380090000068A30033003A00AD
:10564000E200600005003A000003B3003004980057
:10565000110498000080EB002E003700D804900061
:105660000900E00006003A0012002000E680570022
:105670004800900064F807001904980023003700E0
:10568000A80090000100E00008003A00D1A420002A
:1056900021049800010C780021002000510498009A
:1056A000110498000030A000300498001801900008
:1056B000A80090004800900053F8070028009000D0
:1056C0008080EB0011049800AFF897000148780043
:1056D000000CE8002FF89700EA4F50000B003A004A
:1056E000380090000088A3000800320018019000E4
:1056F000A80090004800900043F807000000EB006D
:1057000010049800A8009000010C7800AFF89700F2
:105710000100FB004F04BE000080FA0000000600FC
:1057200000C0DA00000006002800FA00889FBE00D2
:105730008A9FBE008C9FBE0007067800878669009E
:105740000C003B00030478008704780008F0A100F7
:1057500009F0A100840F5000858F5800860F590072
:10576000890F5C00030033000CF0A20001003A0036
:105770000CF0A100EDF807006400E1005F003200CA
:10578000780147006408E100610032006C014700C5
:10579000748557003200BE001201BE003A04BE00FC
:1057A0001A05BE001E039000BE0A90008503530038
:1057B00006003D000004FD008104FD000205FD001F
:1057C0008305FD008703EA00050378000DF8A300B8
:1057D0000400320060041400E0841C0060051D0019
:1057E000E0851D006022B8007D0320000D38E10037
:1057F0008006EB000B0039004433DD00F300B200FB
:105800008301730039003700848272000D02780032
:10581000E10664008B85D1000A85D3008984D3001A
:105820000884D3008703E900F7FF3B00080040002D
:10583000898048000A0149008B81490004003B002F
:1058400060001000E080180060011900E08119007C
:105850000358A300090032008D8272008482720016
:10586000610260008301D1000281D3008180D300F6
:105870000080D3000603E8001B0037000348A300A4
:1058800017003A000600E000170034000603E900A4
:105890000D00A3000000480081804800020149007B
:1058A000838149000348A3000F003A000600E0008E
:1058B000090034000603E900000040008180480030
:1058C000020149008381490001003A000003EB0016
:1058D0000348A300F5FF32006022B8000200370041
:1058E000848272006182660064F8070003F0A10000
:1058F0000CF0A70003F0A000A0F8370064014700F7
:105900006408E10002003A000DF8A30098F83A009C
:105910003200BE001201BE0098F8370000000000FF
:105920008F1FD100780007008F87E9000000E0009A
:1059300000000600809FEB00730007008F87E900DE
:105940000000E00000000600801FEB006E00070072
:105950008F87E9000000E000000006001400FA0054
:10596000889FBE008A9FBE008C9FBE000004BE00C0
:105970000205BE00680047000A90BE000890BE0005
:105980000BF907000070A7000BF0A1000BF8A300B3
:1059900020003A009E0990000E099000FE00900041
:1059A0006E0090009E0290003443200084825200DA
:1059B00072F832000A003C00B4FC2F000428E10019
:1059C000140034008301D1000281D3008180D30010
:1059D0000080D3008502E800FAFF3A0067F837003C
:1059E000B40020000428E10007003C000000400053
:1059F0008180480002014900838149008502E90055
:105A0000FAFF3A005DF8370003002800020020008A
:105A1000010037006011B8006000B80057F8370087
:105A20006011B80019F937001400FA00889FBE0011
:105A30008A9FBE008C9FBE00040678000004BE0052
:105A40000205BE00680047000A90BE000890BE0034
:105A5000D7F807006200E1000800BE000A01BE009E
:105A6000040020000B003A001E029000E43FB10049
:105A70006E009000FE0090000E0990009E099000BC
:105A8000F300B20005FE2300858171000BF0A70032
:105A900003F0A000040E780038F8370007F0A200E9
:105AA00021FF37006022B800060220000000D0006D
:105AB0008180D2000482D2008582D2000000A00042
:105AC0000202520083825A000300310002024200A7
:105AD00083824A000000A1000603E900F3FF3A00B8
:105AE00000000600EFFF07000400BE0000000600F3
:105AF000020AB900001BB9000200B8008100420090
:105B00008100430000000600889FBE008A9FBE00FF
:105B10008C9FBE000404BE000605BE00809FBE0030
:105B2000829FBE0021000700040678000800BE0026
:105B30000A01BE001D000700840678004F03BE0066
:105B40004F02BE008D4F76007FB0970013003300E8
:105B5000F0FF2F008B8F6B0006003B000D066600E8
:105B60000C00A7000A00370007F0A6001000200074
:105B70000A003700880F5200898F5A008A0F5B0095
:105B80008B8F5B00030039001000200001003E00F5
:105B90000000200007F0A7000000EA004F06BE004A
:105BA0004F05BE004F04BE000000060005FF2700A1
:105BB00005826100070032000428E1000100320084
:105BC000240005000600070001003A00440005001B
:105BD0000408050002000700F9FF3A001400050060
:105BE0006F8261008102700085027100850272007F
:105BF000000006001201000000020000000000008A
:105C000000080000D804000055000000010000005A
:105C1000010200000001000009020000290000004C
:105C20000101000000C00000320900000400000073
:105C30000002000003010000010000000921000033
:105C40001101000000010000223F000000070000D9
:105C500005810000030800000001000007050000A6
:105C60000103000008000000010000000403000020
:105C7000090400000A0300004D0000004F0000006E
:105C800047000000490000002A03000075000000E2
:105C90004D0000004F0000004700000049000000D8
:105CA00032000000200000004B00000065000000F2
:105CB00079000000620000006F0000006100000039
:105CC000720000006400000020000000440000009A
:105CD000650000006D0000006F0000000CAE0000C9
:105CE00036AE00003AAE000044AE000005010000F0
:105CF00009060000A10100000507000019E00000EE
:105D000029E70000150000002501000075010000D2
:105D10009508000081020000950100007508000050
:105D200081030000950500007501000005080000D2
:105D300019010000290500009102000095010000F2
:105D4000750300009103000095060000750800002F
:105D5000150000002565000005070000190000007F
:105D60002965000081000000C02500002E320000DF
:105D700066000000506F000074690000203A0000C7
:105D8000202500002E32000066200000560A000088
:105D90003C200000202000003E20000020200000C9
:105DA0002058000020200000204100004443000053
:105DB000000000004B650000796200006F61000088
:105DC0007264000020440000454D00004F0A0000AE
:105DD0003C200000202000003E2000002020000089
:105DE0002058000020200000204100004443000013
:105DF000000000000200FA009EC0A9000080EB0035
:105E0000702488000080EB0050248800AA24EF0052
:105E1000220020008000EB00C04A20004DF807005F
:105E20002000200030258800A824EF008644A90027
:105E3000F009200080248800F009200060248800F8
:105E400082C4A8008804A80000C020004800DE002A
:105E5000C02488000040EB00004F780007003700A6
:105E60001E80FB00C200DD0000C020000081400059
:105E70006000B8000089BE001E4FE8001E40780098
:105E8000E74F5000F6FF36009424A8009624EF0058
:105E900094A4A9009424A900800020005024880024
:105EA00060A020008040EB0001487800C0A02000E6
:105EB0008040EB000148780061508000F00F200026
:105EC00000806000605088007150800000F02F005A
:105ED00000806000705088005024800068006000DE
:105EE0000000E000ECFF3A0010C0B3001BE8B70070
:105EF00010C0B3001CE8B7001D68EF001E68EF007B
:105F00001568EF000040EB00004F780017003700E5
:105F10001E80FB0080004000C08020000080400008
:105F20008000EB00010878001E80FB00800040002C
:105F300080802000008040008000EB000108780095
:105F40009E80FB0020A12000008040008040EB00EC
:105F5000014878009E80FB0040A1200000804000A6
:105F60008040EB00014878001E4FE8001E4078009A
:105F7000E14F5000E6FF360080C0200060408800FE
:105F8000D00020005025880060A12000106088000B
:105F900000C0200081C0B3000148780010C020007C
:105FA00041C0B3000148780010C0200010407800C4
:105FB000804078000174A00010C0200001487800E3
:105FC0000268EF002028EF002228EF002468EF008D
:105FD0000028EF000080FA00000006000200FA002E
:105FE00000408000E10F50000B003A00A124800027
:105FF00000042000008060000000E00006003A007D
:106000000080EB00502488008C04A8008C84A80039
:106010002000200000408800002480007000600004
:106020000000E000070032001024800070006000D3
:106030000000E0000300320000012000002488007E
:10604000BD04070040248000620060000000E00002
:10605000020032008EC0A900A10037005024800049
:10606000610060000000E0000A003200602480004F
:10607000610060000000E000060032005DFF0700E4
:106080009EC0A800400020000040880010002000B2
:106090005024880050248000700060000000E00060
:1060A0000500320060248000700060000000E00005
:1060B0000100320093040700012480000004200046
:1060C000008060000000E0000300320000042000B7
:1060D00000248800F306070050248000640060005C
:1060E0000000E000140032006024800064006000C2
:1060F0000000E00004003200120020008000EB00ED
:1061000030072000750D0700400020005024880053
:1061100019C8BF000004E0000300320019C8BF0026
:106120000040E90019E8B70019C8BF000004E0000A
:1061300001003A00A301070051248000000820005C
:10614000008060000000E000060032006124800052
:1061500000082000008060000000E0000100320024
:106160004C04070050248000620060000000E00042
:106170000C00320060248000620060000000E0003B
:1061800008003200120020008000EB00F0FF270022
:10619000520D07000080EB007024880020002000D2
:1061A0005024880000408000E30F500002003E00B1
:1061B0008EC0A9004A00370060248000680060009B
:1061C0000000E000450032000040EB00004F780086
:1061D0003D00370050248000680060000000E000AF
:1061E0003D003200902480000040780016E8B7009F
:1061F00016C8BF000080FB004400DE0000407800AD
:1062000017E8B700800020005024880016C8BF009F
:10621000684060000004E00011003A0017C8BF00A9
:106220000081FB008080FB0040A120000080400036
:106230009040780061C060000004A200E14060006E
:1062400040A1200000004100E1C060001041780042
:106250000204A1008140710001487800100037005D
:1062600017C8BF000081FB008080FB0020A1200038
:10627000008040009040780061C060000004A200EF
:10628000E140600020A1200000004100E1C060006A
:10629000104178000204A10081407100014878009B
:1062A00017C8BF000004E00002003A002E040700F7
:1062B000040037000001EB0061812000200720006E
:1062C000060D07001E4FE8001E407800E34F500007
:1062D000C0FF360001003700000000008EC0A9009A
:1062E0000080FA00000006000400FA002047980031
:1062F000314798003E4090000080FB00680060003D
:106300000000E000030032008040EB002E409000CF
:106310009B0107003E4090000080FB00640060008D
:106320000000E0000300320011C0B3002E409000D6
:1063300093010700A14A20002E4090000080FB003E
:1063400000004000008F40001E007800BE4090001A
:10635000014878000080FA00000006000800FA00FA
:10636000204798003147980022079800634798001B
:106370003E4090000004E000070032002E409000F4
:106380000080FB0080004000C080200000804000B2
:10639000100F7800060037002E4090000080FB00B0
:1063A000800040008080200000804000100F7800B6
:1063B0001E0078000000E00002003A000000EB0040
:1063C00037003700AE0090001E00780011009800E2
:1063D0001E007800EE409000014878001E00780012
:1063E0001040900002C4B300824060001E0078009C
:1063F000114098001E007800104090008040780006
:106400000134A0001E007800114098001E007800A2
:1064100010409000804078000174A0001E007800B9
:10642000114098003E4090000004E0000E00320051
:106430002E4090000080FB00AE4090008180FB0069
:1064400001814000C180200081004100910078005E
:106450000120A20000014000C08020000000410097
:10646000010878000D0037002E4090000080FB00EE
:10647000AE4090008180FB000181400081802000BF
:1064800081004100910078000120A200000140003D
:106490008080200000004100010878001E00780084
:1064A0000080FA00000006000400FA00204798006F
:1064B000314798002E4090000004E00017003A0099
:1064C0003040800081C0B300014878003040800037
:1064D00061A120001100980030408000C1C0B300CD
:1064E0001140980030408000314080009140900081
:1064F0000174A000114098006040800041C0B300CA
:106500001140980060408000614080009140900000
:106510000174A000114098002E0037002E4090001A
:106520000080FB0000004000800078003E409000AA
:106530000080FB00008040004300DD008000780008
:1065400000C02000008F40001E0078001040900026
:10655000804078000124A0001E00780011409800BF
:106560001E00780010409000804078000174A00068
:106570001E007800114098002E4090000080FB0023
:1065800000004000800078003E4090000080FB004A
:10659000008040004300DD00E400400000C0200017
:1065A000008F40001E00780010409000804078006E
:1065B0000124A0001E007800114098001E00780001
:1065C00010409000804078000174A0001E00780008
:1065D000114098000080FA00000006000200FA0056
:1065E000004F7800A124800000022000008060009D
:1065F0000000E000510032001E80FB0080004000DF
:10660000C080200000804000100278001E80FB0047
:1066100080004000C0802000008040001000780012
:106620001001BE000004200001002000820278005A
:106630000301780080017800010078008382620005
:10664000000061008000EB00C000DD0000002000C1
:106650000001BE006128B800000171008181710055
:10666000028ABE001E80FB0080004000C080200027
:1066700000804000100278001E80FB008000400077
:10668000C080200000804000100078001001BE0093
:1066900000042000010020000000690081806900E2
:1066A000008ABE001E80FB009E80FB00018140002E
:1066B000C180200081004100910078000120A200EB
:1066C00000014000C0802000000041000108780067
:1066D0001E80FB0080004000C08020000080400041
:1066E000900078001E80FB0000014000C080200068
:1066F0000000410010007800104090000044B200FB
:10670000904098001E80FB0080004000C080200068
:1067100000804000900078001E80FB0000014000D7
:10672000C08020000000410010007800104190005F
:1067300000C4B30000406900904098000080FA0057
:10674000000006000000FA009424EF008C24EF0003
:106750000028EF000080FA00000006000000FA00A8
:10676000004080000000E00014003A009424EF0094
:106770008C24EF002000200030258800A824EF00A2
:106780008644A900F009200080248800F009200038
:106790006024880082C4A8009EC0A80001003700C1
:1067A0009404A800A0248000610060000000E000C4
:1067B000FBFF320010002000004088000080FA003B
:1067C000000006000000FA001BC8BF000004A20081
:1067D0000004E0003400320010C0B3001BE8B70032
:1067E0001CC8BF000004A2000004E0002E0032001C
:1067F00010C0B3001CE8B70011C8BF00E24F500042
:106800000C003A00604080008040EB0001487800B6
:106810006040800081C4B300114098006040800057
:1068200061408000914090000174A00011409800E8
:106830001D00370011C8BF00E14F50001A003A0098
:106840001868EF002040800081C0B3000148780044
:106850002040800061A120001100980020408000AD
:1068600041C0B300114098002040800021408000CA
:10687000914090000174A0001140980010C0B30036
:1068800018E8B7003040800081C0B30001487800AC
:106890003040800061A1200011009800304080004D
:1068A00001C8B300114098000080FA000000060003
:1068B0000000FA001D68EF001E68EF0011C8BF005D
:1068C000E24F50000F003A003040800081C0B3001A
:1068D0000148780030408000E1A1200011009800BC
:1068E0003040800081C4B3001140980030408000E7
:1068F00031408000914090000174A0001140980048
:106900001D003700C0A120001080FB00D1A1200095
:106910009180FB00C808DD00010070008000780055
:1069200040508000808F500007003100C0A120003F
:106930001080FB00D1A120009180FB00C808DD0081
:106940000100700040508800960007006040800001
:10695000E1A12000110098006040800081C4B300D4
:10696000114098006040800061408000914090009C
:106970000174A000114098000080FA000000060099
:106980000400FA00204798003147980000C020001A
:10699000000F78002E4090000080FB0000004000B7
:1069A000800078003E4090000080FB0000804000A6
:1069B0004300DD001E0F40001E00780090007800AC
:1069C00001F0A100010878003E4090000004E000C2
:1069D00007003A002E4090000080FB00800040003D
:1069E00080802000008040001E08780006003700EC
:1069F0002E4090000080FB0080004000C0802000FE
:106A0000008040001E0878001E007800900078008A
:106A100001E0A100010878009E0078006480400039
:106A20009000780001E0A000010878000080FA00E2
:106A3000000006000000FA0094A4A9003150800074
:106A400000082000008060000000E00027003A00FD
:106A5000C0A020009040780000C8B30000C06000D3
:106A60000004E0000A00320020C0B30011E8B700C3
:106A70001EC8BF000004A2000004E00001003200B4
:106A80008BFF07001C68EF001B68EF004300370016
:106A90003040800081C0B300014878003040800061
:106AA00061A120001100980030408000C1C0B300F7
:106AB00011409800304080003140800091409000AB
:106AC0000174A000114098006040800041C0B300F4
:106AD000114098006040800061408000914090002B
:106AE0000174A000114098002C00370060A1200024
:106AF0009040780000C8B30000C060000004E000CF
:106B00000F00320010C0B30011E8B7001DC8BF006D
:106B10000004A2000004E0000100320064FF07004E
:106B20001C68EF001B68EF001AC8BF000004A20039
:106B30000004E0001900320022FF070017003700B0
:106B400020C0B30011E8B7003040800081C0B3001E
:106B5000014878003040800061A1200011009800B9
:106B60003040800041C0B3001140980030408000A8
:106B700031408000914090000174A00011409800C5
:106B80001C68EF001B68EF001AC8BF000004A200D9
:106B90000004E000010032000AFF07000080FA0054
:106BA000000006000200FA0080C0B300004F780029
:106BB00040508000E70F50000D003E004050800024
:106BC000004F780010C8BF000004E00003003A0046
:106BD00010C0B30010E8B7000500370010C8BF00B0
:106BE000E14F500002003A0020C0B30010E8B700A7
:106BF000415080001E80FB00008050004050880003
:106C0000604080001E487800E0A12000904088008D
:106C100030508000610060000000E00017003A0082
:106C2000090037009140800020508000104178001A
:106C3000824878008100E800914088000000E80068
:106C4000205088001E4FE9001E4078000004E0003C
:106C5000F4FF3A000C003700914080002050800083
:106C600010417800824878008100E8009140880057
:106C70000000E800205088001E4FE9001E40780008
:106C80000004E000F4FF3A000080FA000000060073
:106C90000200FA0020408000104F78009E80FB0028
:106CA000605080004800DE0073508000F20F20002A
:106CB000028161004811DD0002007000808F5000E9
:106CC00008003600605080004800DE0072508000EE
:106CD000F10F200081006100C808DD000100700094
:106CE000004F7800605080004800DE007250800045
:106CF000F10F200081006100C808DD000100700074
:106D0000800078001E80FB0000805000F10F200002
:106D100081006000C808DD0063508000F20F200091
:106D2000028161008280700061508800C800DE002E
:106D3000F00F2000008060007250800001F02F00F2
:106D40008100610001007000705088000040EB007D
:106D5000104798000C003700505080009E40900073
:106D60000181FB00E1A120008100410091407800F9
:106D7000014878000000E800505088001E40900054
:106D80000040E800104798001E4090009E4F5000C1
:106D9000F1FF3900605080004800DE007250800032
:106DA000F10F200081006100C808DD0001007000C3
:106DB0000000E0001E0032003040800081C0B300BF
:106DC0000148780030408000E1A1200011009800C7
:106DD00020408000900078000000240000806000C7
:106DE0000000E00009003A003040800081C4B30098
:106DF0001140980030408000314080009140900068
:106E00000174A0001140980030003700304080002D
:106E100081C0B300114098003040800031408000B4
:106E2000914090000174A0001140980027003700A5
:106E30003040800081C0B3000148780030408000BD
:106E400061A12000110098003040800041C0B300D3
:106E50001140980030408000314080009140900007
:106E60000174A00011409800705080004800DE00BE
:106E700082508000F10F200081006100C808DD0011
:106E8000010070000000E000080032007050800037
:106E90004800DE0082508000F10F20008100610078
:106EA000C808DD0001007000000001006050800093
:106EB0000070A100605088001AC8BF000004A20042
:106EC0000004E000010032003EFE07000080FA00EE
:106ED000000006000200FA00305080000070A000A0
:106EE00030508800220020008000EB00C04A2000C3
:106EF00018F40700020220008000EB0000C0200010
:106F000014F407009424A8000040EB00004F780020
:106F10000B0037009E80FB0020A120000080400075
:106F20008040EB00014878009E80FB0040A12000DB
:106F3000008040008040EB00014878001E4FE800D0
:106F40001E407800E14F5000F2FF36001200200092
:106F50008000EB0030802000FEF307009424A9009D
:106F600080C020006040880000C0200020408800D1
:106F7000204080003040880080A120001040780030
:106F800002E8B70002C8BF000004E00003003A00B6
:106F90000001200000408800060037001200200099
:106FA0002180200010002000CC09070000022000F2
:106FB000004088000080FA00000006000000FA008F
:106FC00060A120009040780000C8B30080CF50003E
:106FD00047003A0060A0200001CCB30001487800CF
:106FE00090A12000104078000080FB00E20F5000CC
:106FF00009003200E30F500023003200E10F50007F
:1070000037003A00A0DF2A0020508800200120002D
:10701000405088003600370080A1200010407800E2
:107020000004E00014003A0080A120001040780025
:107030000080FB000000400080007800E0E62A00AD
:107040000080400010007800205088002050800010
:107050000080E8009040780080A02000014878007F
:1070600020508000630040009040780090A02000F5
:10707000014878001E00370060A020008040EB002F
:10708000014878001A00370080A1200010407800E5
:10709000E24F50000E003E0080A12000104078001A
:1070A0000080FB00000040008000780000E72A001C
:1070B00000804000100078002050880020508000A0
:1070C000104078000080FB00405088000800370026
:1070D00060A020008040EB000148780004003700E9
:1070E00060A020008040EB00014878000000000014
:1070F0000080FA00000006000200FA00E0A1200073
:107100008040EB0001487800F0A120008040EB00B7
:107110000148780060A12000904078007FC06000A6
:107120000080FB00E10F500011003200E20F500020
:10713000130032000000E00047003A0030508000A9
:107140000070A0003050880014C8BF000004E000A8
:107150003A003200E0A12000104078008040780022
:107160000114A000E0A12000014878003A00370097
:10717000305080000070A00030508800360037008A
:10718000305080000070A00030508800A0A1200086
:10719000104078006F4060000004E00029003200D9
:1071A000A0A120009040780000C8B30000C060009B
:1071B0000004E00009003A00A0A1200090407800FF
:1071C0006FC060000080FB008000400080802000D5
:1071D00000804000100F780008003700A0A12000B8
:1071E000904078006FC060000080FB00800040008D
:1071F000C080200000804000100F78001E00780042
:107200009000780000002800008060000000E0008E
:107210000E0032001E007800900078000040200030
:10722000008060000000E0000A003200E0A12000C1
:1072300011C0B300014878000700370000000000CB
:1072400005003700000000000300370000000000C8
:1072500001003700000000003150800000082000CD
:10726000008060000000E00008003200E0A1200083
:1072700020508800305080000000A000305088006E
:1072800080A0200021C0B300014878000080FA00EF
:10729000000006000000FA00502580006200600037
:1072A0000000E00013003200204080009040900079
:1072B00000C8B30080CF50000D003A00604080004D
:1072C0009040900040C8B30080CF500008003A00C2
:1072D00020408000C1C0B3001140980020408000D1
:1072E00021408000914090000174A000114098005E
:1072F000AA24A90000082000502488000080FA0079
:10730000000006000000FA008284A80000012000AE
:107310005024880010C0B30015E8B7002468EF00BF
:107320000001EB008000EB0050072000EB08070095
:107330000080FA00000006000000FA001568EF0067
:107340000001EB008000EB0040072000E30807008D
:107350008284A90000012000002488002468EF0036
:107360000080FA00000006000000FA00D0C2B3005E
:1073700019E8B70016C8BF000080FB000020A1007C
:107380000000E0001F003A0016C8BF000080FB00AC
:107390004200DE00004078000080FB00C200DD00FB
:1073A00000C0200000804000204088002040800075
:1073B00030408800304080000020A200304088002B
:1073C000204080009000780000C023008080600092
:1073D00000402300808F500008003A0020408000C9
:1073E00010009000820020008000780060A1200042
:1073F000D1F207000B000700080037003D0007002E
:107400000600370016C8BF000080FB000020A10066
:10741000E80F500001003A00530007000080FA0016
:10742000000006000000FA001068EF001A68EF0084
:107430001D68EF001E68EF001868EF001168EF008C
:107440006040800061408000914090000174A10084
:1074500011409800604080000020A2006040880039
:107460006040800061408000914090000174A10064
:1074700011409800604080000020A2006040880019
:107480003040800031408000914090000174A100A4
:107490001140980060A020008040EB000148780077
:1074A0000000EB0040508800C0A020008040EB00AE
:1074B0000148780061508000F00F200000806000DB
:1074C000605088007150800000F02F000080600044
:1074D00070508800830007000001EB008000EB0083
:1074E000300020007D08070052FD07000080FA00F0
:1074F000000006000000FA0011C8BF00E24F500073
:1075000002003A00E2FD0700150037001168EF00A5
:1075100018C8BF000004A2000004E0000F00320001
:107520003040800081C0B3000148780030408000C6
:1075300061A120001100980030408000C1C0B3005C
:107540001140980030408000314080009140900010
:107550000174A00011409800010037001868EF0086
:107560000080FA00000006000200FA00604080007F
:10757000100078004E00DE0061406000004F78008F
:10758000604080000020A200604088000040800031
:10759000E80F50000E003A0080A120001040780053
:1075A0008080FB00F007200000806000B02488008D
:1075B000B02480000000E000030032000001200041
:1075C0000040880002003700400020000040880092
:1075D00011C8BF00E14F500025003A006040800014
:1075E000E1A12000110098006EFD070010C8BF0047
:1075F000E24F500009003A006040800041C0B300F3
:1076000011409800604080006140800091409000EF
:107610000174A00011409800300037001E4078002F
:107620000004E00009003A006040800081C4B3001B
:1076300011409800604080006140800091409000BF
:107640000174A000114098002400370060408000C1
:1076500081C0B3001140980060408000614080000C
:10766000914090000174A000114098001B00370069
:10767000C0A020009040780000C8B30000C06000A7
:107680000004E00014003200705080004800DE006A
:1076900082508000F10F200081006100C808DD00E9
:1076A000010070000000E00008003200705080000F
:1076B0004800DE0082508000F10F20008100610050
:1076C000C808DD000100700000000100605080006B
:1076D0000070A100605088001168EF000080FA007F
:1076E000000006000000FA0060A1200010407800B1
:1076F0000046B2000004E00051003A0070A12000F2
:10770000104078000080FB00CF80DE00B200200037
:1077100003002000820F5000838F58004A003E0073
:1077200000600100210037002200370048003700C8
:107730002000370046003700060037000B003700F6
:107740003A0037000D0037000A0037001B003700F1
:107750002A003700305080000070A00030508800B0
:1077600080002000004088003A00370013FE070028
:1077700038003700D7FD0700360037002080200092
:1077800020508800305080000000A0003050880059
:1077900080A0200011C0B300014878003050800064
:1077A0000070A000305088002A00370052FE070009
:1077B000280037002900070026003700A0A120007C
:1077C000104078008080FB00308020000080400066
:1077D00020508800305080000000A0003050880009
:1077E00080A0200011C0B300014878003050800014
:1077F0000070A00030508800160037003050800024
:107800000070A00030508800A0A120001040780037
:107810000081FB0080A12000904078003080200093
:1078200000004100014878000A0037000001EB0029
:107830008000EB0020002000A807070005003700AB
:1078400000000000030037000000000001003700C6
:10785000000000000080FA00000006000600FA00A8
:1078600080A1200010407800E14F500010003A0045
:1078700060A12000104078007F4060000004E0001C
:107880000B003A00305080000070A000305088009B
:1078900070A1200010407800E34F500003003A0030
:1078A00010C0B30014E8B700010037001468EF00FF
:1078B00080A12000104078000004E000F7003A00AA
:1078C00060A12000104078007F406000E24F50002F
:1078D000F2003A00A0A12000104078006F40600044
:1078E0000004E000ED003200A0A1200090407800EC
:1078F0006FC060000080FB00E10F5000E7003C001B
:107900000140800000022000808F5000E3003A0018
:10791000305080000070A00030508800A0A12000EE
:107920009040780000C8B30000C060000004E00090
:1079300011003A00A0A12000104178006F406100C2
:107940000080FB008000400080802000008040001C
:10795000100F7800A0A12000904078006FC0600058
:107960008080FB0040A12000008040001040780093
:107970004047980010003700A0A120001041780077
:107980006F4061000080FB0080004000C08020004C
:1079900000804000100F7800A0A1200090407800E7
:1079A0006FC060008080FB0020A1200000804000AC
:1079B00010407800404798004E40900061406000C1
:1079C0000004E00004003A001E0078000020A1003E
:1079D000000F7800030037001E0078000020A00090
:1079E000000F7800A0A120009040780000C8B300EC
:1079F00000C060000004E0000A003A00A0A12000DE
:107A0000104178006F4061000080FB009E0078000C
:107A10000001400080802000000041000108780043
:107A200009003700A0A12000904078006FC06000DE
:107A30000080FB009E00780000014000C080200014
:107A4000000041000108780070A12000104078007B
:107A5000E34F50002C003A001E00780090007800A0
:107A600000002800008060000000E00019003200E3
:107A7000A0A120009040780000C8B30000C06000C2
:107A80000004E0000A003A00A0A1200010417800A4
:107A90006F4061008080FB0040A12000008040001A
:107AA000904078000114A0000148780009003700D8
:107AB000A0A12000904078006FC060008080FB0093
:107AC00020A1200000804000904078000114A00018
:107AD000014878001E007800104090008040780037
:107AE0000124A0001E007800114098001E007800BC
:107AF00010409000804078000174A0001E007800C3
:107B000011409800650037001E0078000020A20098
:107B1000000F78001E007800900078000000280018
:107B2000008060000000E000110032001E007800BC
:107B300010409000804078000174A1001E00780081
:107B4000114098001E00780010409000804078009E
:107B50000164A0001E00780011409800220020005F
:107B60009E00780050002000DC0607000600370069
:107B70001E00780010409000804078000164A00052
:107B80001E007800114098001E0078000020A2001E
:107B9000000F78004E409000624060000004E0005A
:107BA00006003A001E0078009000780000002800CF
:107BB000008060000000E00024003200A0A120004E
:107BC0009040780000C8B30000C060000004E000EE
:107BD0000A003A00A0A12000104178006F40610027
:107BE0008080FB0040A12000008040009040780091
:107BF0000114A1000148780009003700A0A120006D
:107C0000904078006FC060008080FB0020A12000C1
:107C100000804000904078000114A10001487800E5
:107C20001E00780010409000B2C3B3008240600094
:107C30001E00780011409800220020009E0078006D
:107C400050002000A5060700060037001E0078003F
:107C500010409000B2C3B300824060001E00780064
:107C600011409800A14A2000A0A1200010417800F6
:107C70006F4061000080FB00000040000080400079
:107C8000100798001E009000104078008040780097
:107C90000114A1001E009000014878000080FA0045
:107CA000000006000000FA00004180001141800041
:107CB00061004000E08048000041880011418800D8
:107CC00015C8BF000004A2000004E0000800320054
:107CD00024C8BF000040E80024E8B70024C8BF0063
:107CE0000004E00002003A0000C0EB0024E8B70006
:107CF0000080FA00000006000400FA000241800043
:107D000013418000028FBE000041800011418000BD
:107D10001E01BE00800F5100818F5900F7FF3A000D
:107D20001E00BE000080FA00000006000000FA00FD
:107D30000000EB0030518800A0A2200041C0B30039
:107D400001487800B0A220008040EB000148780094
:107D5000401F20008041880002003700D041800091
:107D6000A0418800A1418000D0418000808F500058
:107D7000FAFF3A00D1C1B30010C0B3005AF90700AE
:107D800023C0B30042A320008040EB0010C0B3002A
:107D900072F90700405188000080FA0000000600D8
:107DA0006600FA0000408000FF0F500042013600DC
:107DB00040248000620060000000E0000600320005
:107DC00010002000F80507003E013700D041800078
:107DD00090418800010037000000000091418000C0
:107DE000D0418000808F5000F8FF3A009141800020
:107DF000A0418000008F50001E0078000000E000CD
:107E000005003D00A0418000F1FF27008080500068
:107E100090418000008F4000803821009E00780053
:107E2000808F5000040034009141800080C72E00F4
:107E300000804000A0418800305180000000E00038
:107E400006003200305180009000780000002800C9
:107E5000008060000000E00006013A00820020007F
:107E60008000EB00C0A220003AF0070020002000B4
:107E7000CD0507000004E00085003200B0A220001C
:107E8000104078000004A2000004E000C3003200AB
:107E9000B0A2200011C0B3000148780040002000CB
:107EA000AF040700300798003E009000CF80DE004E
:107EB00037EF07006022B800060020000709240001
:107EC00094EE070064662600656626006666260056
:107ED000A700240032EF07004007980051079800E0
:107EE0006207980073079800700047005200200056
:107EF0008000EB0017F00700700047004E02900072
:107F0000DE0290006E039000FE039000849FBE008E
:107F1000869FBE0051EB2A00811F780014F00700F5
:107F2000EA875700760047004E029000DE0290007C
:107F30006E039000FE039000849FBE00869FBE00EB
:107F4000A1EB2A00811F780009F00700EA8757009B
:107F50008000EB0010002000C004070076004700FE
:107F6000010507000000EB00200798000000EB006F
:107F7000200798003C003700F00047002E009000DA
:107F8000008040009040780000C3B30080CF5000D4
:107F900011003400F00047002E00900000804000E7
:107FA0009040780090C3B30080CF50000A003C009E
:107FB000F00047002E009000008040001040780044
:107FC0007340500080407800700147002E00900000
:107FD0000000410001487800F00047002E009000AA
:107FE000008040009040780000C3B30080CF500074
:107FF00005003A00F00047002E009000008040008D
:1080000051C3B30001487800F00047002E009000F3
:108010000080400090407800E0C2B30080CF500064
:1080200005003A00F00047002E009000008040005C
:1080300071C3B30001487800F00047002E009000A3
:108040000080400010407800804078002E019000B1
:10805000E0A2200000004100014878002E009000BE
:108060000000E800200798002E009000E40F500068
:10807000C1FF340030A3200081C2B3000148780062
:10808000605180000010A10060518800430037005B
:1080900010002000440507000004E0000C0032003E
:1080A000B0A22000104078000004A2000004E0000C
:1080B0003A003200B0A2200011C0B300014878009D
:1080C000E0A2200001C5B30001487800330037006A
:1080D00040002000340507000004E0000C003200DE
:1080E000B0A22000104078000004A2000004E000CC
:1080F0002A003200B0A2200011C0B300014878006D
:10810000E0A22000F1C4B30001487800230037004A
:1081100030002000240507000004E0001C003200AD
:10812000B0A22000104078000004A2000004E0008B
:108130001A003200B0A2200011C0B300014878003C
:10814000B04180000000E00009003A00605180006A
:108150000010A00060518800E0A22000E1C3B3003D
:108160000148780010002000B04188000B00370063
:10817000605180000010A10060518800E0A2200042
:1081800091C2B300014878003628EF0003003700A1
:10819000B0A220008040EB00014878000040EB00D6
:1081A000304798000040EB0020479800120037004D
:1081B0002E4090008080FB0060A3200000804000E3
:1081C000904078002E4090000081FB00C0A220006B
:1081D000000041001040780080CF500003003200C2
:1081E00010C0B30030479800060037002E409000C2
:1081F0000040E800204798002E409000E74F5000D4
:10820000EBFF3600804180000000E00006003200F5
:10821000804180009E007800808F50000200350071
:1082200010C0B300304798003E4090000004E000CA
:10823000100032006651800077518000B6518800EE
:10824000C75188008251800093518000D25188002C
:10825000E351880083C0B300C2A2200011C0B30064
:1082600010C0B3003DF807003051880090418000F5
:10827000A0418800405180000000E000060032006C
:1082800040518000900078000000280000806000CD
:108290000000E0000A003A000C00070023C0B30011
:1082A00042A320008040EB0010C0B3002BF8070071
:1082B0004051880003003700000000000100370033
:1082C000000000000080FA00000006000000FA0034
:1082D00040A3200010407800624060000004E000ED
:1082E00003003200300020004E000700020037007B
:1082F000300020007400070040A3200010407800E8
:10830000614060000004E0000300320040002000F3
:108310004400070002003700400020006A00070008
:108320000080FA00000006000000FA00E0A1200032
:108330009040780040A3200001487800E3FF070048
:108340000080FA00000006000000FA00E0A1200012
:10835000F10F200001016000A1A0200091417800F0
:10836000E0C1610002C1710082487800C800DE00EF
:10837000B0A0200010417800604161008140710090
:1083800001487800D0A0200090407800E0C0600054
:108390000134A00001487800E0A02000904078005F
:1083A000E0C060000148780040192400F10F20006F
:1083B00001016000F1A0200091417800E0C161005E
:1083C00002C1710082487800C800DE0000A12000D0
:1083D00010417800604161008140710001487800DF
:1083E000C0A02000904078000174A00001487800EF
:1083F0000080FA00000006000200FA00004F78003A
:10840000114798001E4078000004E00003003A0085
:108410001E4090000080FB00804188000080FA0030
:10842000000006000200FA00000F78001E0078002D
:10843000E40F500018003200E40F500007003E0027
:10844000E20F500010003200E20F500010003E001A
:10845000E10F50000A00320019003700E60F50000B
:1084600011003200E60F50000D003900E70F5000F8
:108470000F003200E80F50000F00320010003700EC
:10848000F4C2A8000E003700F4E2A8000C00370088
:10849000F502A8000A003700F522A80008003700FE
:1084A000F4C2A80006003700F4C2A8000400370098
:1084B000F4C2A80002003700F4C2A80000000000C7
:1084C0000080FA00000006000200FA00000F7800A9
:1084D0001E007800E40F500018003200E40F500036
:1084E00007003E00E20F500010003200E20F500083
:1084F00010003E00E10F50000A0032001900370062
:10850000E60F500011003200E60F50000D00390058
:10851000E70F50000F003200E80F50000F0032004C
:1085200010003700F4C2A9000E003700F4E2A900E1
:108530000C003700F502A9000A003700F522A90057
:1085400008003700F4C2A90006003700F4C2A900F1
:1085500004003700F4C2A90002003700F4C2A900E9
:10856000000000000080FA00000006000200FA008F
:10857000000F78001E007800E40F50003900320030
:10858000E40F500007003E00E20F50001B003200D5
:10859000E20F500026003E00E10F50000A003200BA
:1085A00071003700E60F500048003200E60F50001F
:1085B00039003900E70F500051003200E80F500039
:1085C0005C00320068003700A01780004600DE0023
:1085D000614060000004A200614060000080FB0078
:1085E000610060004600DD00A11780000160A1006D
:1085F00001007000A01788005B003700A017800002
:108600004700DE00614060000004A200614060009D
:108610000080FB00610060004700DD00A1178000C2
:108620000170A10001007000A01788004E00370003
:10863000A01780004800DE00614060000004A20036
:10864000614060000080FB00610060004800DD00C8
:10865000A11780000180A10001007000A017880010
:1086600041003700A01780004900DE006140600033
:108670000004A200614060000080FB006100600017
:108680004900DD00A11780000190A10001007000E9
:10869000A017880034003700A01780004600DE00D5
:1086A000614060000004A200614060000080FB00A7
:1086B000610060004600DD00A11780000160A1009C
:1086C00001007000A017880027003700A017800065
:1086D0004600DE00614060000004A20061406000CE
:1086E0000080FB00610060004600DD00A1178000F3
:1086F0000160A10001007000A01788001A00370077
:10870000A01780004600DE00614060000004A20067
:10871000614060000080FB00610060004600DD00F9
:10872000A11780000160A10001007000A01788005F
:108730000D003700A01780004600DE006140600099
:108740000004A200614060000080FB006100600046
:108750004600DD00A11780000160A100010070004B
:10876000A0178800000000000080FA00000006004A
:108770000200FA00000F78001E007800E40F50009D
:108780002D003200E40F500007003E00E20F5000C1
:1087900017003200E20F50001E003E00E10F5000B3
:1087A0000A00320051003700E60F5000340032005A
:1087B000E60F500029003900E70F50003900320061
:1087C000E80F50004000320048003700A117800039
:1087D000000420000080600000F0A7000000EA0014
:1087E0000000EA004F00DE00004078004000370043
:1087F000A1178000000820000080600000F0A700A2
:108800000000EA000000EA004F00DE0000407800AF
:1088100037003700A11780000010200000806000A2
:1088200000F0A7000000EA000000EA004F00DE00B0
:10883000004078002E003700A117800000202000A3
:108840000080600000F0A7000000EA000000EA00DD
:108850004F00DE000040780025003700A11780009F
:10886000000420000080600000F0A7000000EA0083
:108870000000EA004F00DE00004078001C003700D6
:10888000A1178000000420000080600000F0A70015
:108890000000EA000000EA004F00DE00004078001F
:1088A00013003700A1178000000420000080600042
:1088B00000F0A7000000EA000000EA004F00DE0020
:1088C000004078000A003700A11780000004200053
:1088D0000080600000F0A7000000EA000000EA004D
:1088E0004F00DE0000407800010037000040EB0040
:1088F0000080FA00000006000200FA00000F780075
:108900001E007800E40F500018003200E40F500001
:1089100007003E00E20F500010003200E20F50004E
:1089200010003E00E10F50000A003200190037002D
:10893000E60F500011003200E60F50000D00390024
:10894000E70F50000F003200E80F50000F00320018
:1089500010003700F0C2A9000E003700F0E2A900B5
:108960000C003700F102A9000A003700F122A9002B
:1089700008003700F0C2A90006003700F0C2A900C5
:1089800004003700F0C2A90002003700F0C2A900BD
:10899000000000000080FA00000006000000FA005D
:1089A000A600070014C8BF000004E0000100320068
:1089B00015C8BF000040FE005124800000022000C6
:1089C000008060000000E00002003A0010C0B30028
:1089D00041000700D200070010C0B3000080FA0079
:1089E000000006000000FA0014C8BF000004E00008
:1089F0003600320015C8BF000004E000330032002A
:108A000040248000620060000000E00001003200AD
:108A10008824A900750007000004200000248800B5
:108A2000000000000124800000042000008060009D
:108A30000000E000FBFF320000042000002488005A
:108A4000000000000124800000042000008060007D
:108A50000000E000FBFF320000042000002488003A
:108A6000000000000124800000042000008060005D
:108A70000000E000FBFF32009444A8000004200046
:108A80000024880000000000012480000004200071
:108A9000008060000000E000FBFF320000042000C6
:108AA0000024880000000000012480000004200051
:108AB000008060000000E000FBFF32009444A90049
:108AC0005700070010C0B300010037000040EB0062
:108AD0000080FA00000006000400FA002047980019
:108AE00040248000610060000000E0000B003200C4
:108AF00040248000620060000000E00007003A00AF
:108B000024C8BF00E34F500004003600202480003A
:108B10004300DE0061406000320037002E409000CC
:108B20000004E0001D0032008824A9008804A80089
:108B30002E0007000040EB00004F780009003700CE
:108B400000042000002488000000000001248000B0
:108B500000042000008060000000E000FBFF320005
:108B60001E4FE8001E407800E44F5000F4FF36002E
:108B70000040EB001047980020248000680060004F
:108B80000000E0000200320010C0B300104798005F
:108B9000230007001E409000120037004024800090
:108BA000610060000000E00002003A0000C0EB003D
:108BB0000C00370040248000620060000000E000EC
:108BC00002003A00E0CFB3000600370024C8BF001F
:108BD000E34F500002003E00D0CFB3000100370049
:108BE000C0CFB3000080FA00000006000000FA00C9
:108BF0002E68EF001000FC00F1048000000420004B
:108C0000008060000000E0000200320010C0B300ED
:108C10002EE8B7009EC0A9000080FA000000060000
:108C20000000FA002EC8BF000004E000010032007E
:108C30009EC0A8000080FA00000006000400FA00B0
:108C40001E00FC0011028000000E20000080600069
:108C50003041880011028000000E200001007000E9
:108C60001002880040092000100798000000EB0067
:108C7000000F78000E0037001E0090009000780072
:108C80001E00780000014000E0A320000000410029
:108C9000010878001E0090008000EB0001087800B9
:108CA0001E0090000080E800100798001E0FE800EA
:108CB0001E007800E50F5000EFFF360060248000B2
:108CC000404188008C24EF0010248000504188002F
:108CD0008224EF00700680004800DE0067406000DC
:108CE0000080FB0060418800000120000024880013
:108CF00000022000502488008EC0A9008284A800B1
:108D000071068000F08F2F000080600000A0A0009E
:108D1000700688009EC0A8000080FA0000000600CF
:108D20000400FA0040092000100798000000EB0042
:108D3000000F78000B0037001E0078008000400014
:108D4000E0A3200000804000900078001E0090000A
:108D5000010878001E0090000080E80010079800CD
:108D60001E0FE8001E007800E50F5000F2FF3600ED
:108D70004041800060248800504180001024880019
:108D80006041800000407800674060000080FB0088
:108D9000670060004800DD0072068000F18F2F0040
:108DA00081006100010070007006880011028000DF
:108DB000F0F12F00808060003041800001007000E1
:108DC0003041880030418000100288000080FA00A5
:108DD00000000600040A000022000000000000005D
:108DE000000800002600000000000000000C000049
:108DF00020000000000000003E0A00000C000000FF
:108E000000000000260800000A000000000000002A
:108E10003808000002000000000000003A080000CE
:108E200002000000000000003C08000002000000FA
:108E300000000000260A00001800000000000000EA
:108E40003008000008000000000000009E0900003B
:108E50004000000002000000286E75006C6C2900C4
:108E60000030310032333400353637003839610094
:108E7000626364006566000001000000000A0000F3
:108E80000000640000000000E8030000001027005C
:108E90000000A0008601000040420F000080960004
:108EA00098000000E1F5050000CA9A003B000000B0
:108EB000DE09000026000000020000004B0A00004E
:108EC000004B0A0009000000000200004D0A0000EB
:108ED000004D0A000E02010000000000000000002A
:108EE000000000000602020000000000DE09000091
:108EF0004A0A000006000000000000003E080000D2
:108F000060010000020000000000000000000000FE
:108F1000F03F0000000000000000240040000000BE
:108F20000000000000594000000000000000400068
:108F30008F400000000000000088C30040000000D7
:108F4000000000006AF8400000000000008084007B
:108F50002E41000000000000D0126300410000001C
:108F600000008400D7974100000000000065CD009C
:108F7000CD410000000020005FA0020042408C00B4
:108F8000B5781D00AF154400EA8CA00039593E00A9
:108F90002946A5005CC3F10029633D00489A64009E
:108FA0007EC50E001B514A0044F3C200E4E4E90010
:108FB000634C3D00C7DDD600BA2E77004E5FFB0044
:108FC000F051EF00FC8A5000C7592900090F6B00CF
:108FD0009F527D00C3942500AD49B200545A6200EF
:108FE000D7D71800E77469009C750000883CE4003E
:108FF000377E0000000000000000F0003F9A99005A
:109000009999990099B93F007B14AE0047E17A0025
:10901000843FFC00A9F1D2004D6250003F2D430077
:109020001CEBE200361A3F00F168E30088B5F80057
:10903000E43E8D00EDB5A000F7C6B0003E48AF009D
:10904000BC9AF200D77A3E003A8C3000E28E79006A
:10905000453E9500D626E8000B2E11003EBBBD0014
:10906000D7D9DF007CDB3D00234292000CA19C009D
:10907000C73BA000C2EBFE004B48B400399C570030
:10908000772726006CA137001FB8D4004A7AEE007B
:109090008D352600A6ACAA0004B67900339D3500B4
:1090A0008F1DE9001566310023614D0017ACF800F3
:1090B000522F6F000E998400D94B40002D300500CF
:1090C0008EE42E00FF2B2B00ACF74E0015927E0095
:1090D00068165900F3F8C2001F6EA50001000000D9
:1090E000500A000002000000020000000100000021
:1090F000000000000000FA00F0FC2F00601988005A
:1091000011198000F0FF2100008060001019880014
:1091100025E3A90010C0B30024E3B70021198000A3
:1091200000F0210001007000201988002043A900F0
:1091300001198000000E2000010070000019880055
:1091400021E3A8004119800000FE2F00008060008C
:109150000020A000401988000080FA0000000600EE
:109160000200FA00000F78001E007800004078002E
:109170007F4060000080FB007F006000421980009B
:1091800001FE2F008100610001007000401988007D
:109190002023A8000000000000198000610060008A
:1091A0000000E000FCFF3200001880000080FA00A0
:1091B000000006000000FA000000EB00BD010700FF
:1091C000CCFF07004F000700A0ED2A006600070053
:1091D00008F3070061F50700F1FA0700FEFF37000A
:1091E0000000FA00EC22A8000000000000000000CF
:1091F00000000000EC22A9000080FA000000060038
:109200000000FA000117800000F02F0000806000CD
:1092100000178800F002A900F022A900E822A900A6
:10922000F402A900F422A900EC22A9000080FA00AF
:10923000000006000200FA00004F780021178000AD
:1092400000F02F00808060001E00FB000100700015
:10925000201788000080FA00000006000400FA00D1
:10926000204798003147980001178000F00F200038
:109270000100700000178800F422A800F402A90081
:10928000EC22A80000000000000000000000000028
:10929000101780004700DE0061406000004F78003A
:1092A000EC22A9001E4078000004E000F4FF3A0020
:1092B0000117800000F02F00008060000017880078
:1092C000F422A9003E4090000080FB000000EA006C
:1092D0004F00DE00004078000080FB00610060006D
:1092E000A11780000100A10001007000A0178800F4
:1092F0002E409000CFFF0700B9FF07000080FA0062
:10930000000006000000FA00BDFF07000020210059
:10931000A10720007A0107008040EB0080C3B30062
:10932000CEFF07008040EB0080C0B300CBFF0700FA
:109330008040EB0010C0B300C8FF07008040EB0086
:1093400060C0B300C5FF07008040EB00C0C0B300A1
:10935000C2FF070000B82B000100200068010700D1
:109360000080FA00000006000400FA0010079800D0
:109370000F0037001E009000104F78001E4078004C
:10938000EA4F500004003A008040EB0000CCB300EC
:10939000B2FF0700030037001E40780011C0B30081
:1093A000AEFF07001E0090000000E80010079800C4
:1093B0001E009000104078000004E000EDFF3A002D
:1093C0000080FA00000006000000FA0060A1200002
:1093D000104078007F406000E14F500069003A0083
:1093E000A0A12000104078000004E00067003A00CF
:1093F00070A1200010407800E64F500022003A0093
:1094000090A12000104078000080FB002102200085
:10941000810F50001100320031022000810F5000F6
:109420001600320011022000810F500016003A0091
:1094300002C8BF00E14F500012003A00E0E12A00EC
:1094400020508800900020004050880060A020003C
:1094500001CCB300014878000B00370060E72A0018
:1094600020508800F00320004050880060A02000B9
:1094700001CCB30001487800030037000000000071
:10948000010037000000000060A1200010407800BB
:1094900002C6B3008240600000C2B30080CF50001B
:1094A0003C003A0070A12000104078000080FB00D2
:1094B000E30F500023003200E30F500005003C0092
:1094C000E10F500035003200E20F50000900320079
:1094D00033003700EA0F50000E003200EB0F50004F
:1094E00020003200E90F50002D003A0096FB0700E3
:1094F0002B003700808320002050880010002000BF
:109500004050880060A0200011CCB30001487800D2
:109510002300370060A0200001C8B3000148780094
:1095200090A120001040780038E8B7008183200027
:109530009140780080A1200010407800AEFB070029
:109540001700370090832000205088001000200072
:109550004050880060A0200011C8B3000148780086
:109560000F00370060A0200001C8B3000148780058
:1095700080A120001040780039E8B700000000000A
:109580000700370000000000050037000000000061
:109590000300370000000000010037000000000059
:1095A0000080FA00000006000200FA00000F7800B8
:1095B0001E007800E20F500012003200E20F50004F
:1095C00003003E00E10F5000060032002700370084
:1095D000E30F500014003200E40F50001B00320073
:1095E00022003700901680006200600000F0A700A3
:1095F0000000EA000000E9004F00DE0000407800B3
:109600001B00370011178000002020000080600040
:1096100000F0A7000000EA000000E9004F00DE00B3
:109620000040780012003700111780000010200061
:109630000080600000F0A7000000EA000000E900E0
:109640004F00DE00004078000900370090168000CF
:109650006800600000F0A7000000EA000000E900D8
:109660004F00DE0000407800010037000040EB00B2
:109670000080FA00000006000200FA00000F7800E7
:109680001E007800E20F50000C003200E20F500084
:1096900003003E00E10F5000060032000D003700CD
:1096A000E30F500007003200E40F500007003200C3
:1096B00008003700D022A80006003700E122A800E9
:1096C00004003700E102A80002003700D062A800C1
:1096D000000000000080FA00000006000600FA000A
:1096E000000F780011079800220798001E007800EC
:1096F00021072000810F50002E003200210720009A
:10970000810F50000A003C00E20F50002B00320095
:10971000E20F500003003C00E10F50002100320036
:1097200027003700E30F50002000320024003700EC
:1097300041072000810F5000160032004107200031
:10974000810F50000400350051072000810F5000A8
:109750000C0032001A0037001C000700D1418000C5
:10976000F0FF2700808F500004003200D0418000BD
:109770000000E800D0418800110037003A28EF00CF
:109780000F003700110007001000200049000700FB
:109790000B0037000D0007002000200045000700E7
:1097A0000700370061F907000500370006FF0700D2
:1097B0000300370000000000010037000000000037
:1097C00010C0B3000080FA00000006000000FA009C
:1097D00040248000620060000000E00003003200CE
:1097E0002000200038FB07003000370001408000D7
:1097F00000022000808F500013003A00E0418000FA
:10980000E10F500003003A002000200005FB070094
:1098100023003700E1418000B0042000808F500019
:1098200003003A002000200027FB07001C0037003F
:10983000E141800060092000808F50001500360053
:109840003C28EF0016003700E0418000E10F500097
:1098500003003A0020002000F2FA07001000370051
:10986000E141800020032000808F500003003A0077
:109870002000200014FB070009003700E1418000B0
:10988000603B2000808F5000040036003C28EF0031
:109890000300370000000000010037000000000056
:1098A000E04180000000E800E04188000080FA000C
:1098B000000006000200FA00000F78001E00780089
:1098C000E10F500009003200E10F500009003100A3
:1098D0002000200008FC07003000200006FC0700E4
:1098E0001000200064FF0700030037002BFC070076
:1098F00001003700000000000080FA0000000600B0
:10990000F03FB1000180B10006003500EE03090010
:1099100000000000403FB1000180B100FBFF3D00AE
:109920001000B000203FB0000200350000800900A8
:109930000000000000000600FFFFFF00FFFFFF0027
:020000040001F9
:020000040002F8
:020000040003F7
:020000040004F6
:020000040005F5
:1057F000FFFF0000FFFF0000B62300007F3E000017
:00000001FF
